:0200000480007A
:10000000B72F0000938F0F8073900F306F00400365
:100010001300000013000000130000001300000094
:100020001300000013000000130000001300000084
:100030001300000013000000130000001300000074
:100040009702000093824211739052309300000097
:10005000130100009301000013020000930200004E
:100060001303000093030000130400009304000036
:10007000130500009305000013060000930600001E
:100080001307000093070000130800009308000006
:100090001309000093090000130A0000930A0000EE
:1000A000130B0000930B0000130C0000930C0000D6
:1000B000130D0000930D0000130E0000930E0000BE
:1000C000130F0000930F000097110200938141D19C
:1000D0001705020013050553979503009385457A8C
:1000E00013060000EF00001A170502001305C546AD
:1000F000970502009385854E13060000EF008018D7
:1001000017A503001305057897B503009385457778
:1001100037B6ABAB1306B6BAEF00C01617B1030083
:1001200013014176EF8090609392120093D21200F7
:100130009382D2FF638A02008322010013014100EF
:100140006F0000177300203083220100130141006B
:10015000730020301301C1FF23205100F32220340B
:10016000E3C402FC8322010013014100130141F8A2
:1001700023221100232421002326310023284100BB
:10018000232A5100232C6100232E71002320810299
:10019000232291022324A1022326B1022328C10293
:1001A000232AD102232CE102232EF1022320010570
:1001B0002322110523242105232631052328410567
:1001C000232A5105232C6105232E71052320810745
:1001D000232291072324A1072326B1072328C1073F
:1001E000232AD107232CE107232EF107732520347E
:1001F000F3251034130601006F000000731015344E
:1002000083204100032181008321C10003220101D9
:1002100083224101032381018323C10103240102BD
:1002200083244102032581028325C10203260103A1
:1002300083264103032781038327C1030328010485
:1002400083284104032981048329C104032A010569
:10025000832A4105032B8105832BC105032C01064D
:10026000832C4106032D8106832DC106032E010731
:10027000832E4107032F8107832FC1071301C10775
:10028000730020302320C5006376B50013054500B8
:100290006FF05FFF678000000000000000000000BA
:1002A000000000000000000000000000000000004E
:1002B000130101F8232011002322210023243100FF
:1002C0002326410023285100232A6100232C71009A
:1002D000232E8100232091022322A1022324B10294
:1002E0002326C1022328D102232AE102232CF10272
:1002F000232E010323201105232221052324310568
:100300002326410523285105232A6105232C710545
:10031000232E8105232091072322A1072324B1073F
:100320002326C1072328D107232AE107232CF1071D
:100330009702020083A2822523A02200F322103418
:10034000232E5106EF00C03B1701020003210124B8
:10035000032101008322C10773901234B7220000E9
:100360009382028873A00230832001000322C1001F
:100370008322010103234101832381010324C1015D
:100380008324010203254102832581020326C10241
:100390008326010303274103832781030328C10325
:1003A000832801040329410483298104032AC10409
:1003B000832A0105032B4105832B8105032CC105ED
:1003C000832C0106032D4106832D8106032EC106D1
:1003D000832E0107032F4107832F81071301010893
:1003E00073002030970202009382C22123A01200E2
:1003F00023A2220023A4320023A6420023A85200F5
:1004000023AA620023AC720023AE820023A09202D2
:1004100023A2A20223A4B20223A6C20223A8D202CC
:1004200023AAE20223ACF20223AE020323A01205A8
:1004300023A2220523A4320523A6420523A85205A0
:1004400023AA620523AC720523AE820523A092077E
:1004500023A2A20723A4B20723A6C20723A8D20778
:1004600023AAE20723ACF207EF60D0631701020072
:100470000321C111032101008322C10773901234AB
:10048000B72200009382028873A00230832001000B
:100490000322C1008322010103234101832381013F
:1004A0000324C10183240102032541028325810223
:1004B0000326C10283260103032741038327810307
:1004C0000328C103832801040329410483298104EB
:1004D000032AC104832A0105032B4105832B8105CF
:1004E000032CC105832C0106032D4106832D8106B3
:1004F000032EC106832E0107032F4107832F810797
:100500001301010873002030970202009382820FCA
:1005100083A0020003A1420083A1820003A2C200C3
:1005200083A2020103A3420183A3820103A4C201A7
:1005300083A4020203A5420283A5820203A6C2028B
:1005400083A6020303A7420383A7820303A8C2036F
:1005500083A8020403A9420483A9820403AAC20453
:1005600083AA020503AB420583AB820503ACC20537
:1005700083AC020603AD420683AD820603AEC2061B
:1005800083AE020703AFC20983AF82076780000012
:1005900073700430130101F823201100232221007D
:1005A000232431002326410023285100232A6100FF
:1005B000232C7100232E8100232091022322A102EB
:1005C0002324B1022326C1022328D102232AE102D7
:1005D000232CF102232E01032320110523222105C0
:1005E000232431052326410523285105232A6105AB
:1005F000232C7105232E8105232091072322A10797
:100600002324B1072326C1072328D107232AE10782
:10061000232CF1079702020083A242F723A02200B5
:10062000232E1106EF30406417010200032101F66A
:10063000032101008322C10773901234B722000006
:100640009382028873A00230832001000322C1003C
:100650008322010103234101832381010324C1017A
:100660008324010203254102832581020326C1025E
:100670008326010303274103832781030328C10342
:10068000832801040329410483298104032AC10426
:10069000832A0105032B4105832B8105032CC1050A
:1006A000832C0106032D4106832D8106032EC106EE
:1006B000832E0107032F4107832F810713010108B0
:1006C00073002030737004306F00000073104530E9
:1006D000678000007325403073F04330678000006E
:1006E00097070000938747FE232EB5FE2322C5FA05
:1006F000232635F82320F5F8130505F86780000058
:10070000130101FF23261100EF609036EF20900CBB
:10071000631805008320C1001301010167800000F8
:100720008320C100130101016F300054930785003D
:100730001307F0FF2322F5002324E5002326F5000C
:100740002328F500232005006780000023280500EA
:10075000678000008327450023A2F50003A78700D8
:1007600023A4E50003A787002322B70023A4B70032
:1007700023A8A50083270500938717002320F500F1
:100780006780000003A605009307F0FF13078500AC
:100790006316F6006F008003138707008327470066
:1007A00083A60700E37AD6FE23A2F50023A4B700B0
:1007B00023A4E5002322B70023A8A5008327050072
:1007C000938717002320F5006780000003270501A9
:1007D000832747006FF05FFD0327450083268500D0
:1007E000832705012324D70003278500832645009E
:1007F0002322D70003A747006316A700032785001D
:1008000023A2E7002328050003A507001305F5FF31
:1008100023A0A70067800000032605049387050036
:10082000630406028325C50003274500B385C50080
:100830002326B50063E6E500832505002326B500E1
:10084000138507006F50007F67800000130101FFD0
:100850002324810023261100130405002322910084
:10086000EF30D07483278404635AF0048327440252
:1008700063860704930444026F0000028327840404
:100880009387F7FF2324F404832784046358F0023A
:10089000832744026384070213850400EF3010208D
:1008A000E30E05FCEF30D04C832784049387F7FFD9
:1008B0002324F40483278404E34CF0FC9307F0FF23
:1008C0002324F404EF30D071EF30506E83274404BA
:1008D000635AF00483270401638607049304040128
:1008E0006F000002832744049387F7FF2322F40458
:1008F000832744046358F0028327040163840702BA
:1009000013850400EF309019E30E05FCEF305046DC
:10091000832744049387F7FF2322F40483274404A6
:10092000E34CF0FC9307F0FF2322F404032481003E
:100930008320C10083244100130101016F30506AFC
:10094000630A0508130101FE232C8100130405002E
:10095000232E1100232A910023282101232631016F
:1009600013890500EF309064832404048325C403B5
:100970008329040013850400EF8080351307F0FFFE
:10098000232C0402B3079540B387F9003385A900EF
:100990002322E4042322A400232434012326F40088
:1009A0002324E404631C09028327040163920704DF
:1009B000EF3010638320C1010324810183244101AE
:1009C000032901018329C10013051000130101024D
:1009D00067800000737004306F000000130504018D
:1009E000EFF0DFD413054402EFF05FD46FF05FFC4B
:1009F00013050401EF30900A93071000E31AF5FA8B
:100A0000EFF01FB96FF0DFFA631605007370043062
:100A10006F000000130101FE232A91002328210109
:100A200023263101232E1100232C8100930405007D
:100A300013890500930906006380050AEF804029A9
:100A400013055505EF50803E13040500630E05089D
:100A5000930745052320F500232E94022320240527
:100A6000EF30D054832404048325C40303290400F5
:100A700013850400EF80C0259306F0FF232C0402A9
:100A8000B30795403307A900B307F9002322D40424
:100A90002322E4002326F4002324D40413050401B4
:100AA00023242401EFF09FC813054402EFF01FC870
:100AB000EF30105323083405130504008320C101CF
:100AC0000324810183244101032901018329C100F9
:100AD000130101026780000013054005EF50003547
:100AE0001304050063160500737004306F000000E6
:100AF000232084006FF05FF66316050073700430E6
:100B00006F0000006376B500737004306F00000062
:100B1000130101FF23248100130620001384050024
:100B20009305000023261100EFF01FEE630C050073
:100B3000232C85028320C1000324810013010101BD
:100B400067800000737004306F000000130101FB28
:100B50002326110423248104232291042320210528
:100B6000232E3103232C4103232A5103232861031D
:100B7000232671032326C10063060528638C0526FE
:100B800093072000639CF6000327C503930710001A
:100B90006306F700737004306F00000013890600CD
:100BA0009384050013040500EF309020631A0500BC
:100BB0008327C10063860700737004306F00000054
:100BC000EF30D03E032784038327C403130B0000B8
:100BD000930B20009309F0FF130A0401930A4402C7
:100BE0006364F710630479238327C10063820736A7
:100BF00063160B0013058101EF301005EF30503EF6
:100C0000EF20402FEF30903A83274404639437015C
:100C100023220404832784046394370123240404D7
:100C2000EF30103C9305C10013058101EF30D00473
:100C300063160530EF309037032784038327C403FE
:100C40006304F710EF30D039EF3050368327840437
:100C50006346F0026F00000313850A00EF30006462
:100C600063040500EF30D010832784049387F7FFD7
:100C70002324F404832784046356F000832744026A
:100C8000E39C07FC23243405EF309035EF3010321D
:100C9000832744046346F0026F00000313050A0033
:100CA000EF30C05F63040500EF30900C83274404ED
:100CB0009387F7FF2322F404832744046356F0004C
:100CC00083270401E39C07FC23223405EF305031D5
:100CD000EF20C055130B1000EF30502D0327840375
:100CE0008327C403E370F7F00326040463040612A9
:100CF000631A091E0325840093850400EF50803396
:100D0000832784008326040403274400B387D70085
:100D10002324F40063E4E71083278403832604007C
:100D200003274402938717002324D400232CF402C2
:100D30006300071013054402EF304056930710007C
:100D40006318F50E6F004014EF3090298325C10021
:100D500013050A00EF308027EF30502583278404E5
:100D60006346F0026F00000313850A00EF30005362
:100D700063040500EF30C07F832784049387F7FF67
:100D80002324F404832784046356F0008327440259
:100D9000E39C07FC23243405EF309024EF3010212E
:100DA000832744046346F0026F00000313050A0022
:100DB000EF30C04E63040500EF30807B832744048E
:100DC0009387F7FF2322F404832744046356F0003B
:100DD00083270401E39C07FC23223405EF305020D5
:100DE000EF20C044E31805EEEFF08FFA130B10006C
:100DF0006FF09FEE83270504E38407D873700430F7
:100E00006F000000737004306F00000003260404BC
:100E1000631006088327040063860704832784037E
:100E20000327440293871700232CF402E31407F0EE
:100E3000EF30101B130510008320C104032481042C
:100E400083244104032901048329C103032A810364
:100E5000832A4103032B0103832BC10213010105E4
:100E60006780000003254400EF3050078327840388
:100E7000032744022322040093871700232CF40243
:100E8000E31A07EAE30605FAEFF08FF06FF05FFA76
:100E90000325C40093850400EF50C0198327040480
:100EA0000327C40083260400B307F0403307F7008C
:100EB0002326E400637ED70403274400B307F7002A
:100EC0002326F40013072000832744026304E90467
:100ED0000327840313071700232CE402E38A07F493
:100EE0006FF05FE50325C40093850400EF50801484
:100EF000832704040327C40083260400B307F040BB
:100F00003307F7002326E400E37ED7FA6FF0DFFA19
:100F10008327440203278403E30C07FA032784038F
:100F20001307F7FF232CE40203278403130717009A
:100F3000232CE402E38E07EE6FF0DFDF13050400DD
:100F4000EFF0DF90EF20802E130500006FF0DFEE52
:100F5000EF301009130500006FF01FEE130101FFC1
:100F600023229100930405001305400523248100EA
:100F700023261100EF40906B13040500630C050459
:100F8000232C05029307F0FF2322F504130710001A
:100F900013050501232EE4022324F4042322040074
:100FA0002320040023240400232604002320040417
:100FB00023089404EFF08FF713054402EFF00FF7C6
:100FC00093060000130600009305000013050400BB
:100FD000EFF0DFB7130504008320C1000324810074
:100FE00083244100130101016780000063040504AC
:100FF000130101FF232481002322910023261100E5
:10100000232021010329450013040500EF30405936
:10101000930400006304A9028320C100032481001B
:1010200013850400032901008324410013010101F9
:1010300067800000737004306F0000008327C400D5
:10104000930410009387F7FF2326F400E39607FC30
:10105000930600001306000093050000130504002A
:10106000EFF0DFAE6FF05FFB130101FC232E1102E6
:10107000232C8102232A91022328210323263103D2
:10108000232441032326C100630E050A93090000AF
:10109000638405101389060093840500130405007A
:1010A000130A05016F008003EF308073EF3000708A
:1010B0009305C10013058101EF30003C6310050664
:1010C000EF30C06E032784038327C403630CF70249
:1010D000EF300071EF30C07093091000EF30006DF9
:1010E000032784038327C4036362F7068327C100B1
:1010F00063860702E39A09FA13058101EF30C034D1
:101100006FF09FFAEF30C06D8325C10013050A0010
:10111000EF20D06BEFF0CFC76FF0DFFBEF30406C0C
:101120008320C10303248103832441030329010392
:101130008329C102032A810213050000130101045F
:1011400067800000737004306F0000000326040401
:101150006314060683270400638807048327840337
:101160000327440293871700232CF4026310070817
:10117000EF3000678320C1030324810383244103EC
:10118000032901038329C102032A810213051000E8
:10119000130101046780000083270504E38C07EE38
:1011A000737004306F00000003254400EF300053DB
:1011B000232204006FF09FFA6316090403258400BC
:1011C00093850400EF40106783278400832604047E
:1011D00003274400B387D7002324F400E3E0E7F8B3
:1011E000832704002324F4006FF05FF71305440203
:1011F000EF30C00A93071000E31CF5F6EFF04FB98B
:101200006FF01FF70325C40093850400EF40906240
:10121000832704040327C40083260400B307F04097
:101220003307F7002326E4006378D7000327440040
:10123000B307F7002326F40093072000E310F9F228
:1012400083278403E38C07F0832784039387F7FFC6
:10125000232CF4026FF09FF0130101FC232E1102E6
:10126000232C8102232A91022328210323263103E0
:10127000232441032326C1006308051493040000BE
:10128000638C051293890600138905001304050079
:10129000130A45026F000001EF308054EF304054D4
:1012A00093041000EF30805083278403639E070867
:1012B0008327C100638C070463840404EF30405229
:1012C000EF30C04E9305C10013058101EF30C01A05
:1012D000631E0502EF30804D83278403E39E07FAE7
:1012E000EF30005083270400638607048325C10084
:1012F00013050A00EF20904DEFF08FA96FF01FFA51
:1013000013058101EF3040146FF05FFBEF30404D6B
:101310008320C103032481038324410303290103A0
:101320008329C102032A810213050000130101046D
:1013300067800000EF30804703254400EF30002A2B
:10134000EF30004A6FF09FFA032604048324C400A0
:101350006304060203274400B387C4002326F40075
:1013600063E6E700832704002326F4008325C400F6
:1013700013050900EF40104C639C09048327840384
:10138000032704009387F7FF232CF402631607005A
:10139000EF30404C2322A40083270401638007041C
:1013A00013050401EF20906F930710006318F502F6
:1013B000EFF00F9E6F00800283270504E38407ECA3
:1013C000737004306F000000737004306F00000011
:1013D000832744022326940063960702EF3040409F
:1013E0008320C103032481038324410303290103D0
:1013F0008329C102032A810213051000130101048D
:101400006780000013054402EF205069E30805FCE3
:101410006FF01FFA6302050A63880508130101FED5
:10142000232C8100232A9100232821012324410118
:10143000232E1100232631019307200093840600F8
:1014400013090600138A050013040500639CF600C7
:101450000327C503930710006302F70A7370043073
:101460006F000000EFF00FA7032784038327C40356
:10147000930905006366F7049304000013850900CF
:10148000EFF0CFA48320C101032481011385040060
:1014900003290101832441018329C100032A81001A
:1014A000130101026780000083270504E38807F623
:1014B000737004306F000000737004306F00000020
:1014C00003260404631E060C8327040063860712A8
:1014D000832784031307F0FF93871700232CF4025C
:1014E000832784046388E70E832784049304100011
:1014F000938717002324F4046FF05FF8EFF08F9DBB
:10150000032784038327C403930905006360F70658
:1015100003260404E30A06FA0325C40093050A001F
:10152000EF405031832704040327C40083260400BE
:10153000B307F0403307F7002326E4006378D700B1
:1015400003274400B307F7002326F4009307200085
:10155000E390F4F883278403E38C07F6832784035E
:101560009387F7FF232CF4026FF09FF60326040401
:10157000E30C06F40325C40093050A00EF40902B0A
:10158000832704040327C40083260400B307F04024
:101590003307F7002326E400E364D7FA6FF09FFBDC
:1015A000E39C04F60325840093050A00EF4090288D
:1015B000832784008326040403274400B387D700CD
:1015C0002324F400E3E6E7F0832704002324F40057
:1015D0006FF01FF08327440293041000E38007EAB2
:1015E00013054402EF20904BE30A05E8E30809E8FD
:1015F000232099006FF09FE803254400EF30000E90
:10160000232204006FF0DFEC6302050A8327050440
:1016100063860700737004306F00000083270500A5
:10162000638A0708130101FE232C8100232A9100FD
:10163000130405002328210123263101232E110044
:1016400013890500EFF00F89032784038327C40360
:1016500093090500930400006376F702832784034F
:101660001307F0FF93871700232CF40283278404C9
:10167000638AE70483278404930410009387170088
:101680002324F40413850900EFF04F848320C10163
:1016900003248101138504000329010183244101EE
:1016A0008329C100130101026780000073700430B8
:1016B0006F00000083274500E38607F6737004304F
:1016C0006F00000083274402639607009304100014
:1016D0006FF05FFB13054402EF20503CE30805FE6A
:1016E000E30609FE930710002320F9006FF01FFEA8
:1016F000130101FC232E1102232C8102232A9102C3
:1017000023282103232631032324410323225103C9
:101710002326C10063060528638C0526938A0600EC
:101720009389050013040500EF209068631A0500F3
:101730008327C10063860700737004306F000000C8
:10174000EF30C006832784036394071C8327C100FE
:101750006380071013058101EF20104F9304F0FF01
:1017600013094402130A0401EF308007EF10807858
:10177000EF30C003832744046394970023220404BA
:10178000832784046394970023240404EF304005E6
:101790009305C10013058101EF20104E631005244D
:1017A000EF30C00083278403638A070AEF304003C9
:1017B000EF20D07F832784046346F0026F0000038C
:1017C00013050900EF20902D63040500EF20505A07
:1017D000832784049387F7FF2324F4048327840456
:1017E0006356F00083274402E39C07FC23249404FF
:1017F000EF20107FEF20907B832744046346F002A4
:101800006F00000313050A00EF2050296304050050
:10181000EF201056832744049387F7FF2322F40414
:10182000832744046356F00083270401E39C07FCEC
:1018300023229404EF20D07AEF10501FEF2010776E
:10184000832784036396070C8327C100E39E07F078
:10185000EF201079130500006F00800FEF20507803
:1018600083270400638807108325C100130509003E
:10187000EF20C075EF209073832784046346F00245
:101880006F00000313050900EF20502163040500D9
:10189000EF20104E832784049387F7FF2324F4045A
:1018A000832784046356F00083274402E39C07FCEB
:1018B00023249404EF20D072EF20506F8327440438
:1018C0006346F0026F00000313050A00EF20101DAD
:1018D00063040500EF20D049832744049387F7FF72
:1018E0002322F404832744046356F0008327040171
:1018F000E39C07FC23229404EF20906EEF1010135A
:1019000063040508EF20906A83278403E38E07F2BF
:1019100093850900130504008324C400EFE0DFEF82
:1019200063940A0883278403032704009387F7FF3F
:10193000232CF40263160700EF20D0712322A400A9
:101940008327040163920708EF20906913051000B4
:101950008320C1030324810383244103032901035A
:101960008329C102032A8102832A4102130101044F
:1019700067800000EF20906303254400EF201046AD
:10198000EF2010666FF05FEEEFE09FC06FF09FF703
:1019900083270504E38407D8737004306F000000C8
:1019A000737004306F0000008327440223269400E4
:1019B000E38C07F813054402EF20500EE30605F808
:1019C000EFE01FBD6FF05FF813050401EF20100D6D
:1019D00093071000E31AF5F66FF09FFE130504005D
:1019E000EFE0DFE6EF109004130500006FF05FF604
:1019F00063000506130101FF232481002320210138
:101A00002326110023229100832445001389050019
:101A100013040500EF20D0386380A404930600006F
:101A2000130609009305000013050400EFF05FCCD6
:101A300093071000630CF5028320C100032481008A
:101A40008324410003290100130101016780000084
:101A5000737004306F0000008327C400130510006A
:101A6000938717002326F4006FF01FFD8327C4001F
:101A7000938717002326F4006FF01FFC6308050608
:101A80006386050C130101FE232C8100232A91009B
:101A900023282101232631012324410113040500B9
:101AA000232E11001309060093890500EFE09FC261
:101AB00083278403130A050093040000639C070234
:101AC00013050A00EFE09FC08320C10103248101B8
:101AD0001385040003290101832441018329C100E6
:101AE000032A810013010102678000007370043033
:101AF0006F00000003260404630406028325C4006B
:101B000083274400B385C5002326B40063E6F500AF
:101B1000832504002326B40013850900EF4080517B
:101B2000832784031307F0FF9387F7FF232CF40226
:101B3000832744046384E70283274404930410004A
:101B4000938717002322F4046FF09FF7832705047F
:101B5000E38A07F2737004306F00000083270401EA
:101B600063960700930410006FF09FF513050401BE
:101B7000EF20C072E30805FEE30609FE930710009C
:101B80002320F9006FF01FFE630605088327050474
:101B9000638A050863840708130101FE232C810072
:101BA000232A910023282101232441011304050045
:101BB000232E110023263101138A0500EFE09FB187
:101BC000832784031309050093040000638E070034
:101BD0008329C40093050A0013050400EFE0DFC366
:101BE000930410002326340113050900EFE01FAE13
:101BF0008320C1010324810113850400032901010D
:101C0000832441018329C100032A810013010102B9
:101C100067800000737004306F0000007370043040
:101C20006F000000E38C07FE737004306F0000004B
:101C300063160500737004306F000000130101FF8C
:101C4000232481001304050023261100EF20103601
:101C500003248403EF20D0388320C100130504003F
:101C60000324810013010101678000006316050051
:101C7000737004306F000000130101FF2326110070
:101C80002324810013040500EF20503283278403AE
:101C90000324C4033304F440EF20903413050400FC
:101CA0008320C1000324810013010101678000002B
:101CB0006306050003258503678000007370043008
:101CC0006F0000006308050497870300938787B7B8
:101CD00003A747006304E50403A7C7006302E50800
:101CE00003A74701630AE50603A7C7016302E506E8
:101CF00003A74702630AE50403A7C7026302E504DA
:101D000003A74703630AE50203A7C7036302E502CB
:101D10006F40C029737004306F000000130700008B
:101D200013173700B387E70023A007006F40002890
:101D3000130770006FF0DFFE130760006FF05FFEA7
:101D4000130750006FF0DFFD130740006FF05FFDD9
:101D5000130730006FF0DFFC130720006FF05FFC0B
:101D6000130710006FF0DFFB0325C5046780000038
:101D70002326B50467800000034505056780000041
:101D800063080500032585031335150067800000EF
:101D9000737004306F000000630C05008327850317
:101DA0000325C5033305F540133515006780000092
:101DB000737004306F00000097870300938787A833
:101DC00003A707006300070403A78700630807044D
:101DD00003A707016308070403A787016308070433
:101DE00003A707026308070403A787026308070421
:101DF00003A70703630C070403A78703630407040F
:101E0000678000001307000013173700B387E7004F
:101E100023A0B70023A2A7006780000013071000CB
:101E20006FF09FFE130720006FF01FFE13073000B6
:101E30006FF09FFD130740006FF01FFD1307500068
:101E40006FF09FFC130770006FF01FFC130760001A
:101E50006FF09FFB978703009387C79E03A74700F8
:101E60006300E50403A7C7006306E50403A7470171
:101E70006306E50403A7C7016306E50403A7470259
:101E80006306E50403A7C7026306E50403A7470347
:101E9000630AE50403A7C7036302A7046780000081
:101EA0001307000013173700B387E70023A00700CC
:101EB00067800000130710006FF0DFFE130720009B
:101EC0006FF05FFE130730006FF0DFFD1307400077
:101ED0006FF05FFD130750006FF0DFFC1307700019
:101EE0006FF05FFC130760006FF0DFFB130101FF71
:101EF00023248100232291002320210113040500C3
:101F0000232611009384050013090600EF20100A10
:101F1000032744049307F0FF6314F700232204040B
:101F2000032784049307F0FF6314F70023240404B9
:101F3000EF20100B83278403639A07001306090020
:101F40009385040013054402EF208024EF2010063F
:101F500083278404635AF0048327440263860704BA
:101F6000930444026F000002832784049387F7FFE1
:101F70002324F404832784046358F0028327440253
:101F80006384070213850400EF204031E30E05FC53
:101F9000EF20005E832784049387F7FF2324F40453
:101FA00083278404E34CF0FC9307F0FF2324F4041C
:101FB000EF201003EF20807F83274404635AF0044E
:101FC0008327040163860704930404016F00000261
:101FD000832744049387F7FF2322F40483274404D0
:101FE0006358F00283270401638407021385040009
:101FF000EF20C02AE30E05FCEF208057832744041E
:102000009387F7FF2322F40483274404E34CF0FC76
:102010009307F0FF2322F404032481008320C100EE
:102020008324410003290100130101016F20407B3B
:1020300063020504130101FD232E3101232C41010C
:1020400023261102138A07002324810223229102EE
:1020500023202103232A5101232861012326710112
:10206000930790009309070063FAE7007370043048
:102070006F000000737004306F000000130B050048
:102080009384050013090600938B0600930A080049
:102090006302082C13050006EF30505913040500A5
:1020A0006302052A13192900232855031306090082
:1020B0009305500A13850A00EF40C00903C70400C6
:1020C000832704031309C9FF230AE40203C704009A
:1020D000338927011379C9FF6306070E83C71400EC
:1020E000A30AF40283C71400638E070C83C724007D
:1020F000230BF40283C724006386070C83C73400D4
:10210000A30BF40283C73400638E070A83C744001D
:10211000230CF40283C744006386070A83C7540074
:10212000A30CF40283C75400638E070883C76400BE
:10213000230DF40283C764006386070883C7740015
:10214000A30DF40283C77400638E070683C784005F
:10215000230EF40283C784006386070683C79400B6
:10216000A30EF40283C79400638E070483C7A40000
:10217000230FF40283C7A4006386070483C7B40057
:10218000A30FF40283C7B400638E070283C7C400A1
:102190002300F40483C7C4006386070283C7D40006
:1021A000A300F40483C7D400638E070083C7E40050
:1021B0002301F40483C7E4006386070083C7F400A7
:1021C000A301F404930A440013850A00A301040444
:1021D0002326340323283405232A0404EFE00FD7F1
:1021E00013058401EFE08FD69307A000B387374132
:1021F000232C040423288400232CF40023228402AB
:1022000023220404232E040413860B0093050B00E1
:1022100013050900EFE0CFCC2320A40063040A00DB
:1022200023208A007370043017E901001309493430
:102230008327090097E4010093844435638C0700E9
:1022400003A7040083A7040083274704938717008C
:102250002322F70417E701001307473283270700FB
:102260009387170097E6010023AAF63083A704009E
:10227000638E070E8327090017EB0100130B4B40F9
:10228000639C070083A7040083A7C70263E6F900E5
:1022900097E7010023AC872E97E701009387472C2F
:1022A00083A7070017E701001307C72C0325C40203
:1022B000032707009387170097E6010023A2F62A59
:1022C0002324F4046376A70097E7010023A4A72A38
:1022D00093054001EF60D01F93850A003305AB00E2
:1022E000EFE04FC7832709006388070083A7040036
:1022F00083A74704639C0708832709001304100081
:10230000638A070083A7040083A7C70263F4370129
:10231000EFE00FA8130504008320C102032481020B
:1023200083244102032901028329C101032A810177
:10233000832A4101032B0101832BC10013010103F7
:102340006780000013850A00EF3050461304F0FF49
:102350006FF05FFC13152600EF30502D930A050037
:10236000E31A05D21304F0FF6FF0DFFA97E70100DC
:1023700023AE87200327070093071000630AF702A4
:1023800017EB0100130BCB2F6FF01FF103A7040015
:1023900083A60400832747049387F7FF2322F704CB
:1023A00083A74604E39A07F4736004306FF0DFF408
:1023B000130A000017EB0100130B8B2C930BA000EA
:1023C00013050A0093054001EF609010130A1A00EC
:1023D0003305AB00EFE08FB5E3147AFF97EB010014
:1023E000938B8B3613850B00EFE04FB417EA010097
:1023F000130ACA3613050A00EFE04FB317E50100D0
:1024000013050537EFE08FB217E501001305853797
:10241000EFE0CFB117E5010013050538EFE00FB18C
:1024200097E7010023A2771797E7010023AC471530
:102430006FF09FE6130101FF232481002326110082
:10244000232291002320210113040500737004301E
:1024500097E401009384C41183A70400639E0710CE
:102460006318040097E701009387471203A407004D
:102470001309440013050900EFE00FB68327840217
:102480006386070013058401EFE00FB5930509008B
:1024900017E501001305052FEFE0CFAB97E701002B
:1024A0009387070E03A7070097E701009387470B61
:1024B00083A707001307170097E6010023A2E60C85
:1024C00003A704009387170097E6010023AAF608E4
:1024D000630C070097E701009387470B03A70700EA
:1024E00003274704631C070E83A70400638A0706BB
:1024F00097E701009387870903A707006302871006
:102500007370043003A704006318070817E701007D
:10251000130787078326070083A606006392060A2F
:102520001307F0FF97E6010023AAE60203A70400C1
:102530006308070203A70700032747046302070293
:1025400003A7070083A60700832747049387F7FFA5
:102550002322F70483A746046394070073600430C2
:102560008320C1000324810083244100032901004A
:10257000130101016780000097E7010093870701BD
:1025800003A7070083A70700832747049387170043
:102590002322F7046FF0DFEC83A6070003A70700F0
:1025A00003A746041307170023A2E60417E7010058
:1025B000130787FD8326070083A60600E38206F63D
:1025C000032707000327C7000327C7000327470087
:1025D00097E6010023A4E6F86FF05FF503A7070074
:1025E00083A60700832747049387F7FF2322F70476
:1025F00083A74604E39A07EE736004306FF0DFEEC2
:1026000097E70100938747F583A7070063860700D4
:10261000737004306F000000032481008320C10028
:102620008324410003290100130101016FD05FF6EB
:102630006304050C17E70100130747F5832607001D
:10264000930700006386A60A130101FF23261100E9
:1026500023248100232291007370043097E6010047
:10266000938606F183A70600638C07000326070004
:102670008327070083274604938717002322F60445
:1026800083A706009304050003244501638807001F
:102690008327070083A747046394070697E7010091
:1026A000938787EE83A70700638C870697E701006F
:1026B000938747ED83A707006384870697E70100A8
:1026C0009387870D6306F40497E701009387870BD0
:1026D000630CF402930710008320C10003248100DF
:1026E0008324410013850700130101016780000066
:1026F0001385070067800000737004306F000000CE
:10270000EF6000736FF09FF9930740006FF0DFFCFC
:1027100083A7840293B71700938727006FF0DFFB2E
:10272000930720006FF05FFB7370043097E70100A0
:10273000938707E403A707006316070263040504F1
:1027400083A707000325C502638C070097E70100F4
:102750009387C7E303A7070003274704631C070207
:102760006780000017E70100130747E28326070090
:102770000327070003A746041307170023A2E60454
:10278000E31005FC17E70100130747E003250700E6
:102790006FF01FFB03A7070083A6070083274704EA
:1027A0009387F7FF2322F70483A74604E39A07FAE7
:1027B0007360043067800000130101FF232481004F
:1027C0001304050023261100EFD0DFF06318040086
:1027D00097E70100938787DB03A407000324C40263
:1027E000EFD0DFEE8320C100130504000324810035
:1027F00013010101678000009307900063F6B700A2
:10280000737004306F000000130101FE232C81005F
:10281000232E1100232A9100232821012326310190
:1028200023244101130405007370043017E90100EB
:10283000130909D483270900639207106300041267
:1028400083270405638EF50A17E70100130707D4F1
:1028500063F0B70283260700638E86120327070002
:102860008324C702B3B4950093C414006F00000121
:1028700083240700B384844093B414000327C40264
:102880006386E70E832784012328B40463C8070006
:102890009307A000B385B740232CB40093172700FB
:1028A000B387E7000327440197E90100938949DDD5
:1028B00093972700B387F9006310F704130A4400C5
:1028C00013050A00EFD05FF197E70100938787CAED
:1028D0000325C40283A7070063F6A70097E701005A
:1028E00023AAA7C893054001EF60803E93050A0024
:1028F0003385A900EFD01FE663840400EFD05FC9E1
:1029000083270900638C070097E70100938707C8B6
:1029100083A7070083A74704639E07048320C101A0
:102920000324810183244101032901018329C1007A
:10293000032A8100130101026780000097E701006C
:102940009387C7C403A7070083A70700832747040B
:10295000938717002322F704E31404EE97E701009E
:102960009387C7C203A407006FF09FED2326B4022C
:102970006FF05FF1032481018320C10183244101B1
:10298000032901018329C100032A810013010102E7
:102990006F60004A930400006FF05FEE630A050861
:1029A000130101FE232A910097E40100938404BEE1
:1029B00083A70400232E1100232C8100232821014A
:1029C000232631016388A7047370043017E90100DE
:1029D000130909BA83270900638C070003A70400C1
:1029E00083A7040083274704938717002322F70453
:1029F0000327450197E70100938707DA630EF70283
:102A0000832709006388070083A7040083A747047E
:102A1000639E07088320C1010324810183244101AF
:102A2000032901018329C10013010102678000000D
:102A3000737004306F0000008327850217E70100E0
:102A4000130707D3E38EE7FAE39C07FA93094500DF
:102A50001304050013850900EFD01FD897E7010084
:102A6000938747B10325C40283A7070063F6A70035
:102A700097E7010023A0A7B093054001EF60402530
:102A800097E701009387C7BF3385A70093850900A7
:102A9000EFD05FCC83A704000327C40283A7C7023B
:102AA000E360F7F6EFD0DFAE6FF09FF5032481010E
:102AB0008320C10183244101032901018329C1002D
:102AC000130101026F60C03663020506130101FEA7
:102AD000232C8100232A91002326310113040500B1
:102AE000232E110023282101EFD0DFBE032744014C
:102AF00097E70100938747CA9309050093040000F4
:102B0000630AF70213850900EFD05FBC8320C1017F
:102B10000324810113850400032901018324410159
:102B20008329C10013010102678000007370043023
:102B30006F0000008327840217E50100130545C3D9
:102B4000E382A7FCE39007FC97E701009387C7A007
:102B500083A707006394070697E70100938707A3FD
:102B600083A707008324C4021309440083A7C70274
:102B700013050900B3B4F400EFD01FC697E70100B6
:102B80009387479F0325C40283A7070093C41400BB
:102B900063F6A70097E7010023AEA79C93054001C9
:102BA000EF60001397E70100938787AD9305090055
:102BB0003385A700EFD01FBA6FF0DFF493058401CF
:102BC000EFD05FB96FF01FF4130101FE371500005D
:102BD000232E1100232C8100232A91002328210178
:102BE00023263101232441012322510123206101A5
:102BF000EF30C02363080522930405001305000687
:102C0000EF30C022130405006304052637160000C8
:102C10009305500A2328950213850400EF30805352
:102C200083240403B71700009387C7FFB384F4001D
:102C3000B7474C4593879744130A4400232AF4026C
:102C400013050A00230C0402A30104042326040232
:102C500023280404232A0404EFD05FAF1305840162
:102C6000EFD0DFAE9307A000232C040493F4C4FF3D
:102C700023288400232CF40023228402232204042A
:102C8000232E040413060000971500009385C5EA5F
:102C900013850400EFD0DFA42320A4007370043058
:102CA00017E901001309C98C8327090097E4010083
:102CB0009384C48D638C070003A7040083A70400DA
:102CC00083274704938717002322F70417E701009F
:102CD0001307C78A832707009387170097E6010029
:102CE00023AEF68883A704006388070A83270900B8
:102CF00097E901009389C998639C070083A70400A2
:102D000083A7C7026396070097E7010023A087887F
:102D100097E701009387C78403A7070097E60100A0
:102D2000938646858327C40283A6060013071700EF
:102D300017E601002326E6822324E40463F6F60066
:102D400017E701002328F782139527003305F500C4
:102D50001315250093050A003385A900EFD09F9F26
:102D6000832709006388070083A7040083A747041B
:102D7000639E070C832709006384070083A7040070
:102D8000EF20500793071000630AF510631C050835
:102D9000737004306F00000097D7010023A8877E6E
:102DA000032707009307100097E901009389498DD5
:102DB000E310F7F6938A090017EB0100130BCB9889
:102DC00013850A00938A4A01EFD05F96E31A5BFFEE
:102DD00017E5010013054597EFD05F9597EA0100CD
:102DE000938ACA9713850A00EFD05F9417E5010014
:102DF00013050598EFD09F9317E5010013058598FB
:102E0000EFD0DF9217E5010013050599EFD01F926F
:102E100097D7010023AA677797D7010023A4577794
:102E20006FF01FEF8320C10103248101832441013E
:102E3000032901018329C100032A8100832A41005B
:102E4000032B0100130101026780000003A70400A7
:102E500083A60400832747049387F7FF2322F70400
:102E600083A74604E39807F0736004306FF09FF087
:102E7000032481018320C101032901018329C100A9
:102E8000032A8100832A4100032B010013850400DB
:102E900083244101130101026F304011737004302B
:102EA0009307F0FF17D70100232AF76A0324810153
:102EB00097D7010023AEA76A8320C1018324410173
:102EC000032901018329C100032A8100832A4100CB
:102ED000032B010097D7010023A0076A1301010209
:102EE0006FD04FD07370043097D7010023A20768CA
:102EF0006FD08FE117D701001307076683270700FC
:102F0000938717002320F700678000007370043058
:102F100097D701009387C76503A7070063180702C7
:102F200017D70100130747650325070083A707008C
:102F3000638C070097D701009387476503A70700B5
:102F400003274704631407026780000017D70100B6
:102F50001307C763832607000327070003A7460458
:102F60001307170023A2E6046FF09FFB03A70700D7
:102F700083A60700832747049387F7FF2322F704DC
:102F800083A74604E39207FC736004306780000067
:102F9000130101FF2326110023248100EFD08FF3BA
:102FA00097D701009387475D03A40700EFD00FF286
:102FB0008320C100130504000324810013010101D3
:102FC0006780000097D701009387475B03A5070040
:102FD00067800000130101FD2326110223248102D2
:102FE0002322910223202103232E3101232C41018E
:102FF000232A5101232861012326710197D701005B
:103000009387875583A70700639A070617D70100A0
:1030100013078756832707009387170097D6010069
:1030200023ACF654832A0700638A0A0A97D7010063
:103030009387C75283A707009304000063FEFA0A30
:1030400097D901009389C96317DA0100130A0A545A
:1030500083270A009306100003A7C70293172700CF
:10306000B387E70093972700B389F90083A7090086
:1030700063F4F602930410006F00000297D701007A
:103080009387C74E83A70700930400009387170018
:1030900017D70100232CF74C97D701009387C74C13
:1030A00083A7070063840700930410008320C102F4
:1030B00003248102138504000329010283244102B1
:1030C0008329C101032A8101832A4101032B0101C4
:1030D000832BC100130101036780000017D4010096
:1030E0001304844A8327040083A707006388070C1E
:1030F000737004306F00000017D401001304C4483B
:1031000097D901009389C95717DA0100130A0A48B1
:1031100017DB0100130B0B468327040083A707006E
:10312000638007088327040083A7C70003A9C7009B
:1031300083274900930B490013850B0063EAFA06C5
:10314000EFD08FE983278902130589016384070083
:10315000EFD08FE88327C90203270B0093850B006C
:10316000139527003305F500131525003385A900B5
:103170006376F70017D70100232EF73EEFD08FDDDF
:1031800083270A000327C90283A7C702E366F7F86B
:10319000832704009304100083A70700E39407F833
:1031A0009307F0FF17D70100232AF73A6FF05FEA81
:1031B00017D701002324F73A6FF09FE917D70100D2
:1031C0001307473C832704000327070097D6010015
:1031D00023ACE63A17D701002326F73A97D7010028
:1031E0009387473883A707009387170017D70100F5
:1031F000232AF7368327040083A70700639A070072
:103200009307F0FF17D70100232AF7346FF01FE26E
:103210008327040083A7C70083A7C70083A74700AD
:1032200017D70100232CF7326FF05FE097D701002A
:103230009387873203A70700631607007370043073
:103240006F000000130101FE232E1100232C8100CA
:10325000232A91002328210123263101232441011F
:1032600023225101232061017370043097D401009F
:103270009384043003A704006310071203A7070018
:103280001307F7FF97D6010023A8E62C83A70700B2
:10329000639E070A97D701009387472E83A70700ED
:1032A0006386070A97DA0100938A8A3D17DA0100DC
:1032B000130A4A2C17D901001309492D930910004C
:1032C0006F00C0013385EA00EFD0CFC88327090023
:1032D0000327C40283A7C7026374F70683A70A0FF4
:1032E0006380070E83A7CA0F03A4C70013058401D8
:1032F000EFD08FCE130B440013050B00EFD0CFCDD2
:103300008327C40283260A0093050B001395270028
:103310003305F50013152500130705003385AA00B2
:10332000E3F2F6FA17D701002326F724EFD08FC275
:10333000832709000327C40283A7C702E360F7FAC3
:1033400097D7010023A237236FF05FF91304000021
:1033500083A70400638C070097D701009387072396
:1033600083A7070083A74704639807041305040095
:103370008320C10103248101832441010329010128
:103380008329C100032A8100832A4100032B010005
:10339000130101026780000017D701001307071F00
:1033A000832607000327070003A746041307170017
:1033B00023A2E6046FF09FECEF5090276FF01FFB05
:1033C00017D401001304841A83270400638C0702B6
:1033D000832704001309100063860702EFF09FBFE4
:1033E0006306050097D7010023A02719832704004F
:1033F0009387F7FF17D70100232AF71683270400C6
:10340000E39E07FC97D701009387071603A70700E1
:1034100093071000E31CF7F2EFD08F97130410000E
:103420006FF01FF3630405026396050073700430A8
:103430006F00000017D7010013070712832707004A
:10344000638A0700737004306F00000073700430EB
:103450006F000000130101FF2324810023261100C7
:1034600083260700032705009386160017D6010060
:103470002324D60E97D601009386061083A6060055
:103480003304B7002320850063F0E6046372E4028E
:1034900063F0860297D701009387470F03A50700C3
:1034A00013054500EFD04FB313050400EF50D00FC4
:1034B000EFF0DFD7630E05008320C10003248100F5
:1034C0001301010167800000E366E4FC6FF05FFC1C
:1034D000032481008320C100130101016FD04F8BB1
:1034E000630E050017D7010013070707832707009E
:1034F00063880700737004306F0000006FD04F893D
:10350000130101FF23261100232481000327070054
:10351000930705001307170097D6010023AEE602B4
:1035200097D601009386860617D701001307C704B4
:103530000327070003A506003304F7001305450021
:10354000EFD08FA913050400EF501006EFF01FCE47
:10355000631A0500032481008320C10013010101C7
:103560006FD00F838320C100032481001301010168
:1035700067800000130101FF23248100232611002E
:1035800097D70100938747FD83A707001304000026
:103590009387170017D701002320F7FC97D7010066
:1035A0009387C7FD83A7070063EEF51417DE0100BC
:1035B000130ECE1897D201009382C20B13040000A1
:1035C00013070000930F10001303500A6F00C00090
:1035D000130ECEFE6384C20F83278EFF930607006F
:1035E000E38807FE8327CEFF83A74700232EFEFE36
:1035F0006386C71303AFC70083A747003307E500FF
:10360000930E0000232EFEFE6380C70983A8C70027
:1036100093874803232017012322F70083A78804F8
:103620002326F7012324F70083A7C8022328F700E5
:1036300083A70805232C0700232AF70003A8080303
:10364000834708006398670493070800938717006F
:1036500083C60700B3850741E38A66FE93D525003C
:103660009395050193D50501231EB700938E1E0087
:1036700013070702630A1F038327CEFF83A74700B0
:10368000232EFEFEE394C7F983274E00232EFEFE71
:103690006FF0DFF793050000231EB700938E1E0026
:1036A00013070702E31A1FFD3304D4011317540054
:1036B000130ECEFE93060700E390C2F397D70100E6
:1036C000938787EC03AE070083270E0063960712EB
:1036D00097D70100938707EB03AE070083270E00FF
:1036E000639A071C17DE0100130E8EF983274E1014
:1036F000639C070283278E11639C072663040600E0
:1037000023200600EFF09FB2130504008320C100C0
:1037100003248100130101016780000083274E000C
:10372000232EFEFE6FF01FED83278E1017DF0100A2
:10373000130FCF0583A7470017D701002326F704EF
:103740006386E73D83A2C70083A74700B306D50081
:10375000930E000017D701002328F702930F4000B3
:103760001303500A6382E70983A8C70093874803BD
:1037700023A0160123A2F60083A7880423A6F6013E
:1037800023A4F60083A7C80223A8F60083A7080590
:1037900023AC060023AAF60003A808038347080009
:1037A000639A6732930708009387170003C70700DF
:1037B000B3850741E30A67FE93D725009397070176
:1037C00093D70701239EF600938E1E009386060270
:1037D000638C123183278E1083A7470017D701000F
:1037E0002324F7FAE392E7F983270E1117D7010094
:1037F000232CF7F86FF05FF783274E00130F8E002E
:1038000083A647002322DE006380E633B307E5008A
:1038100003A7460083A2C600930E00002322EE00F9
:10382000930F20001303500A6300EF088328C7009A
:103830001387480323A0170123A2E70003A78804E6
:1038400023A6F70123A4E70003A7C80223A8E700E3
:1038500003A7080523AC070023AAE70003A8080371
:1038600003470800631E67221307080013071700A9
:1038700083460700B3050741E38A66FE13D7250098
:103880001317070113570701239EE700938E1E00AD
:10389000938707026380122383264E0003A7460006
:1038A0002322EE00E314EFF80327CE002322EE00DC
:1038B0006FF0DFF783274E00130F8E0083A74700BA
:1038C0002322FE00638CE72583A2C70083A747005D
:1038D000B306D500930E00002322FE00930F2000B4
:1038E0001303500A6300FF0883A8C70093874803A7
:1038F00023A0160123A2F60083A7880423A6F601BD
:1039000023A4F60083A7C80223A8F60083A708050E
:1039100023AC060023AAF60003A808038347080087
:1039200063986714930708009387170003C707007D
:10393000B3850741E30A67FE93D7250093970701F4
:1039400093D70701239EF600938E1E0093860602EE
:10395000638A121383274E0083A747002322FE00A9
:10396000E314FFF88327CE002322FE006FF0DFF779
:103970008327CE1197DE0100938E8EE283A7470046
:1039800017D70100232CF7E0638AD71783AFC7004E
:1039900083A747003307D5001303000097D6010023
:1039A00023AEF6DE130F3000930220009308500A76
:1039B0006388D70903A5C700930745032320A70001
:1039C0002322F700832785042326E7012324F70019
:1039D0008327C5022328F700832785026384070015
:1039E0002326570083270505232C0700232AF700E9
:1039F0000328050383470800639C17059307080005
:103A00009387170083C60700B3850741E38A16FF33
:103A100093D725009397070193D70701231EF7003B
:103A20001303130013070702638EAF028327CE111F
:103A300083A7470097D6010023A2F6D6E39CD7F7C9
:103A400083274E1297D6010023AAF6D46FF09FF673
:103A500093070000231EF700130313001307070248
:103A6000E396AFFC33046400E31C06C86FF09FC903
:103A700093070000239EF600938E1E009386060295
:103A8000E39A12ED17DE0100130E8EBF83274E104E
:103A90003304D40193165400E38E07C46FF0DFC8DB
:103AA00013070000239EE700938E1E0093870702F2
:103AB000E39412DF97D701009387C7AC03AE0700EA
:103AC0003304D4019316540083270E00E38C07C0FF
:103AD0006FF05FDE93070000239EF600938E1E00BA
:103AE00093860602E39812CF83278E113304D40104
:103AF00093165400E38407C06FF09FE783274E12AC
:103B000017D70100232CF7C86FF05FE883270E1149
:103B100017D70100232AF7C66FF0DFC28327CE0034
:103B20002322FE006FF05FDA8326CE002322DE0020
:103B30006FF0DFCD130101FD232291022320210329
:103B4000232E3101232C4101232A51012328610115
:103B500023267101232611022324810297D9010013
:103B60009389899F17D90100130989B117DA0100D8
:103B7000130A0AA097DA0100938A4AA197DB010091
:103B8000938BCB9F97D401009384849F130B1000D9
:103B90006F00000283A709000324491093871700D0
:103BA00017D70100232AF79AEFF04FE8631E0400AD
:103BB00083A70400E39007FE83270900E37AFBFE56
:103BC000EFC01F9D6FF0DFFE7370043083270A0083
:103BD000639E07048327091103A4C700130544004B
:103BE000EFC09FBF83A70B009387F7FF17D7010094
:103BF0002326F79883A704009387F7FF17D70100C0
:103C00002320F79883270A006388070083A70A0008
:103C100083A747046398070203250403EF200039B4
:103C200013050400EF2080386FF09FF803A70A0007
:103C300083A70A0083274704938717002322F704EA
:103C40006FF05FF903A70A0083A60A0083274704E1
:103C50009387F7FF2322F70483A74604E39E07FA1E
:103C6000736004306FF05FFB97D701009387C78EB6
:103C700083A70700639E070E130101FF232611008F
:103C8000232481002322910097D7010023AE078CC3
:103C900017D701001307878F83270700B7A6A5A5AD
:103CA0009386565A83A7070383A50700639ED50012
:103CB00003A64700631AB60083A687006396C60072
:103CC00083A7C700638AD700032507008325070061
:103CD00093854503EF30007717D7010013078789D5
:103CE0008326070017D40100130484996F00000293
:103CF0008327070063860708832707009387F7FF5A
:103D000097D6010023A8F6868326070093972600FE
:103D1000B387D70093972700B307F40083A7070062
:103D2000E38807FC0325070093172500B387A70046
:103D3000939727003307F400832647009387870073
:103D4000B307F40083A4460023229700638EF40295
:103D500083A7C4008320C1000324810017D701007A
:103D60002326F782832441001301010167800000AC
:103D70009307100017C701002328F77E6780000013
:103D8000737004306F00000083A444009305400169
:103D9000EF4010743305A400232295006FF05FFB01
:103DA000130101FE23282101232E1100232C810061
:103DB000232A910023263101130905007370043072
:103DC00097C401009384C47A83A7040017C4010038
:103DD0001304C47B639C070C6314090003290400CB
:103DE0009309490013850900EFC01F9F83278902AB
:103DF0006386070013058901EFC01F9E93850900A4
:103E000017D5010013054599EFC0DF9483A704007F
:103E1000638807008327040083A747046394070A85
:103E2000832704006384270D83A7040063820706A9
:103E30007370043083A704006398070E97C70100CE
:103E40009387877403A70700032707006310070CF5
:103E50009307F0FF17C701002322F77083A7040020
:103E6000638807028327040083A74704638207024D
:103E70000327040083260400832747049387F7FF62
:103E80002322F70483A74604639407007360043079
:103E90008320C101032481018324410103290101FD
:103EA0008329C10013010102678000000327040079
:103EB0008327040083274704938717002322F704EE
:103EC0006FF09FF103270400832604008327470433
:103ED0009387F7FF2322F70483A74604E39207F4AE
:103EE0007360043083270400E39027F583A7040060
:103EF0006382070697C701009387076683A70700B9
:103F00006388070A737004306F00000083A70700FE
:103F100083A7C70083A7C70083A7470017C701006F
:103F2000232EF7626FF09FF303270400832704001A
:103F300083274704938717002322F70497C70100BC
:103F40009387876403A7070003270700E30207F0AE
:103F50006FF0DFFB97C701009387476217C7010027
:103F60001307077283A70700032787116314F7025B
:103F70008320C1010324810197C7010023A80760A2
:103F800083244101032901018329C1001301010296
:103F900067800000032481018320C1018324410143
:103FA000032901018329C100130101026FF0DFCB56
:103FB000032481018320C1018324410103290101DC
:103FC0008329C100130101026FC08FDC6306050A5B
:103FD000130101FF2322910097C401009384045B25
:103FE000232021011389050083A504002326110045
:103FF0002324810093858501EFC0CFF803A5040039
:1040000013054500EFC04FFD9307F0FF630AF90663
:1040100097C701009387475603A4070003A704002E
:1040200083A707003304240123228700636EF4066C
:1040300097C701009387475503A5070083A5040090
:1040400093854500EFC00FF497C701009387075190
:1040500083A707006376F40097C7010023A0875069
:104060008320C1000324810083244100032901002F
:104070001301010167800000737004306F000000BD
:1040800083A50400032481008320C1008324410010
:104090000329010017C5010013050570938545002C
:1040A000130101016FC00FEB97C701009387874D84
:1040B00003A507000324810083A504008320C10019
:1040C0008324410003290100938545001301010168
:1040D0006FC04FEB630E050097C701009387C7477A
:1040E00083A70700639A0700737004306F00000015
:1040F000737004306F000000130101FF2322910050
:1041000097C401009384844803A7040093870500A3
:1041100083A50400B7060080B3E7D700232611006B
:1041200023248100232CF7009385850113040600C6
:10413000EFC04FE203A5040013054500EFC0CFE92F
:104140009307F0FF6304F40297C701009387C74207
:1041500003A507008320C1008324410033058500A7
:1041600003248100130101016F40104483A5040062
:10417000032481008320C1008324410017C501006E
:104180001305856193854500130101016FC08FDC24
:104190006308050A130101FF2322910097C401005F
:1041A0009384C43E232021011389050083A50400C4
:1041B0002326110023248100938585011304060022
:1041C000EFC04FD903A5040013054500EFC0CFE0B1
:1041D00093071000630AF40697C701009387C73955
:1041E00003A4070003A7040083A7070033042401E6
:1041F00023228700636EF40697C701009387C738B0
:1042000003A5070083A5040093854500EFC08FD761
:1042100097C701009387873483A707006376F4006C
:1042200097C7010023AC87328320C100032481009B
:10423000832441000329010013010101678000006C
:10424000737004306F00000083A504000324810014
:104250008320C100832441000329010017C5010008
:104260001305855393854500130101016FC08FCE5F
:1042700097C701009387073103A507000324810036
:1042800083A504008320C100832441000329010089
:1042900093854500130101016FC0CFCE130101FFCB
:1042A0002326110023248100232291008327C500A7
:1042B00003A4C7006304040A930484011385040063
:1042C000EFC08FD197C701009387072983A7070005
:1042D000639A07089304440013850400EFC0CFCF0E
:1042E00097C70100938707290327C40283A7070004
:1042F00063F6E70097C7010023AEE7269317270070
:10430000B387E7009397270017C5010013054537CA
:10431000938504003305F500EFC0CFC397C70100B4
:104320009387C72683A707000327C402130500004D
:1043300083A7C70263FAE7009307100017C70100BD
:104340002324F722130510008320C10003248100D9
:104350008324410013010101678000007370043061
:104360006F0000009385040017C501001305454048
:10437000EFC04FBE6FF09FFA97C701009387C71D2C
:1043800083A7070063960700737004306F00000076
:10439000130101FF23261100232481002322910011
:1043A000B70700800324C500B3E7F5002320F5001C
:1043B00063080408EFC04FC293044400138504004F
:1043C000EFC08FC197C701009387C71A0327C402A4
:1043D00083A7070063F6E70097C7010023ACE7183F
:1043E00093172700B387E7009397270017C50100AD
:1043F000130505293305F50093850400EFC08FB53B
:1044000097C701009387871883A707000327C40273
:104410001305000083A7C70263FAE70093071000A3
:1044200017C701002322F714130510008320C100D1
:1044300003248100832441001301010167800000EF
:10444000737004306F0000006304050297C7010019
:104450009387471103A7070097C701009387C711E8
:1044600083A707002320E5002322F50067800000D2
:10447000737004306F0000006304050E638E050C3A
:10448000130101FF232611002324810013070500D7
:104490007370043097C801009388880D83A70800C3
:1044A0006380070297C701009387470E83A6070022
:1044B00083A7070083A746049387170023A2F60467
:1044C00017C301001303430B83A705000326030052
:1044D0009306F0FF130400006388D70417CE010091
:1044E000130E4E0803250E000328070083264700FD
:1044F0006306A800130410006378D6023308D64080
:10450000130410006372F80203250E00B387C7403E
:1045100003260300B387D70023A0F5002320A700BC
:104520002322C7001304000083A70800638C070040
:1045300097C701009387870583A7070083A74704D0
:1045400063940702130504008320C1000324810043
:104550001301010167800000737004306F000000D8
:10456000737004306F000000EF40900C6FF09FFDFF
:104570009307100017C701002328F7FE678000008B
:10458000630605000325C5046780000013050000CD
:1045900067800000630405002326B50467800000DF
:1045A00097C70100938787FE03A507006780000077
:1045B00097C701009387C7FB83A707001305100067
:1045C000638C070097C70100938707F903A50700CD
:1045D000133515001315150067800000630C0508DE
:1045E000130101FE232A910097C40100938404FA69
:1045F00083A70400232E1100232C810023282101EE
:10460000232631010327C50283A7C7026376F70477
:104610008327850163CC070083A7040083A6C70214
:104620009307A000B387D740232CF50093172700EA
:10463000B387E7000327450117C90100130949049F
:1046400093972700B307F9006308F70283A70400D4
:1046500083A7C7022326F5028320C1010324810119
:1046600083244101032901018329C10013010102AF
:10467000678000006780000093094500130405006F
:1046800013850900EFC04F9583A7040017C70100E9
:10469000130747EE0327070083A7C7022326F40268
:1046A0006376F70017C701002326F7EC1395270060
:1046B0003305F50003248101131525008320C10172
:1046C00083244101938509003305A9008329C10092
:1046D00003290101130101026FC0CF8763060502A0
:1046E000130101FF232611002324810023229100BE
:1046F00097C70100938787E903A40700630AA40012
:10470000737004306F000000130500006780000024
:104710008327440563960700737004306F00000020
:104720008326C402032704059387F7FF232AF40492
:104730006384E600638E0700130500008320C10038
:1047400003248100832441001301010167800000DC
:104750009304440013850400EFC00F88032504056B
:1047600097C70100938707E103A707009307A000FD
:10477000B387A7402326A402232CF4006376A70066
:1047800097C7010023A8A7DE93054001EF404054DE
:1047900097C701009387C7EE3385A7009385040070
:1047A000EFB05FFB130510006FF05FF9737004301A
:1047B00097C701009387C7DB83A7070063800702C1
:1047C00097C70100938787DC03A7070083A707002B
:1047D00083274704938717002322F704678000008C
:1047E00097C701009387C7D883A70700638C070288
:1047F00097C70100938787D903A7070003274704BA
:104800006302070203A7070083A607008327470464
:104810009387F7FF2322F70483A7460463940700D6
:10482000736004306780000097C70100938707D644
:1048300003A6070083A6070003A707009307A000AD
:1048400083A6C60203258601B387D740232CF70031
:104850006780000097C70100938747D303A707002D
:10486000630A070083A6070003A74605130717007E
:1048700023AAE60403A5070067800000130101FDD9
:1048800023202103232611022324810223229102C3
:10489000232E3101130905007370043097C4010001
:1048A000938404CD83A7040017C40100130404CE2D
:1048B000639E070A8327040083A78705639A07007E
:1048C000832704001307100023AEE704639A050E44
:1048D00083A70400638807008327040083A7470495
:1048E000639A07147370043083A704006394070667
:1048F0008327040003A587056308050063020904F4
:104900008327040023AC07048327040023AE070495
:1049100083A70400638807008327040083A7470454
:10492000639207068320C10203248102832441028B
:10493000032901028329C1011301010367800000DB
:1049400003270400832787059387F7FF232CF704A9
:104950006FF09FFB0327040083270400832747048D
:10496000938717002322F7046FF09FF803270400B2
:104970008327040083274704938717002322F70423
:104980006FF05FF3032704008326040083274704A6
:104990009387F7FF2322F70483A74604E39407F8DD
:1049A000736004308320C102032481028324410206
:1049B000032901028329C10113010103678000005B
:1049C000032504002326B10013054500EFB0DFE006
:1049D0008325C1009307F0FF6380F50897C70100A6
:1049E000938787B983A907000327040083A70700DB
:1049F000B389B9002322370163ECF90697C7010098
:104A0000938787B803A50700832504009385450095
:104A1000EFB05FD797C70100938747B483A707001C
:104A200063F6F90097C7010023AA37B3EFB05FB66A
:104A30006FF01FEA0327040083260400832747043E
:104A40009387F7FF2322F70483A74604E39C07E834
:104A5000736004306FF01FE98325040017C501005F
:104A6000130585D393854500EFB0DFCE6FF01FFCB3
:104A700097C70100938707B103A5070083250400AA
:104A800093854500EFB01FD06FF05FFA130101FD71
:104A900023202103232E3101232611022324810206
:104AA00023229102232C410113890500930906005A
:104AB0007370043097C40100938484AB83A704000F
:104AC00017C40100130484AC639C0714032704007B
:104AD000930720000327C7056304F7028327040018
:104AE0001345F5FF03A787053375E50023ACA7043D
:104AF000832704001307100023AEE704639A060A15
:104B000083A70400638807008327040083A7470462
:104B1000639407167370043083A70400639E07062E
:104B2000638809008327040083A7870523A0F90071
:104B30000327040093071000130500000327C7058F
:104B4000630EF700832704001349F9FF13051000D3
:104B500003A787053379E90023AC270583270400E1
:104B600023AE070483A7040063880700832704009B
:104B700083A747046392070C8320C10203248102A8
:104B800083244102032901028329C101032A8101EF
:104B9000130101036780000003270400832704003A
:104BA00083274704938717002322F7046FF05FF7EA
:104BB000032504002326D10013054500EFB0DFC113
:104BC0008326C1009307F0FF638AF60C97C70100A4
:104BD0009387879A03AA07000327040083A7070087
:104BE000330ADA00232247016368FA0C97C70100F1
:104BF0009387879903A507008325040093854500C3
:104C0000EFB05FB897C701009387479583A7070068
:104C10006370FA0A97C7010023A247956F00400905
:104C20000327040083270400832747049387170082
:104C30002322F7046FF09FE9032704008326040072
:104C4000832747049387F7FF2322F70483A74604AB
:104C5000E39407F2736004308320C10203248102CD
:104C600083244102032901028329C101032A81010E
:104C7000130101036780000003270400832604005A
:104C8000832747049387F7FF2322F70483A746046B
:104C9000E39207E8736004306FF0DFE783250400D8
:104CA00017C50100130545AF93854500EFB09FAAD6
:104CB000EFB01F8E6FF0DFE497C701009387878CFA
:104CC00003A507008325040093854500EFB09FAB43
:104CD0006FF01FFE630A050C130101FF232611006C
:104CE00023248100232291002320210173700430AA
:104CF00097C401009384C48783A7040063960708C0
:104D0000638606008327850523A0F6009307060027
:104D1000930620000326C505232ED504138705001E
:104D2000130405006382D70A63F4F6089305300084
:104D30006388B700930540006396B700630CD610F4
:104D4000232CE40493071000630CF60813041000EE
:104D500083A70400638C070097C70100938707832C
:104D600083A7070083A74704639807061305040079
:104D70008320C10003248100832441000329010012
:104D8000130101016780000097C701009387078026
:104D900003A7070083A7070083274704938717000B
:104DA0002322F7046FF0DFF5737004306F0000000A
:104DB00093061000E398D7F88327850533E7B700FB
:104DC000232CE5046FF01FF88327850593871700D0
:104DD000232CF5046FF01FF7EF4080056FF01FF9EB
:104DE0001309440013050900EFB01F9F97B7010096
:104DF000938747780325C40283A7070063F6A700BB
:104E000097B7010023A8A77693054001EF30506CB7
:104E100097C701009387C7863385A70093050900CC
:104E2000EFB05F93832784026386070073700430BA
:104E30006F00000097B701009387477583A70700AD
:104E40000327C40283A7C702E3F2E7F0EFB04FF4F1
:104E50006FF0DFEF130400006FF09FEF63080508A9
:104E6000130101FE232C8100232A91002328210114
:104E7000232631012324410123225101232E110035
:104E800093090700138A060093040600138905009E
:104E900013040500EFB01F84930A050063060A009F
:104EA000832784052320FA000327C40593072000E5
:104EB000232EF4046380F40463FA97109306300001
:104EC0006388D400930640006396D400630CF70E09
:104ED000232C2405930710006312F70A832784020A
:104EE00063820702737004306F0000007370043037
:104EF0006F0000008327840593871700232CF40498
:104F00006FF05FFD97B701009387076583A70700E0
:104F10006390070A9304440013850400EFB0DF8B0D
:104F200097B70100938707650325C40283A707008D
:104F300063F6A70097B7010023AEA762930540016F
:104F4000EF30105997B7010093878773938504005A
:104F50003385A700EFB01F8097B7010093870763E1
:104F600083A707000327C40283A7C70263F8E700EB
:104F7000638609009307100023A0F90013041000B2
:104F800013850A00EFB08FF4130504008320C101DC
:104F90000324810183244101032901018329C100E4
:104FA000032A8100832A4100130101026780000067
:104FB0009305840117B501001305857BEFB08FF9C8
:104FC0006FF09FF9130400006FF09FFB9307100030
:104FD000E392F4F08327840533E92701232C240589
:104FE0006FF05FEF630A050E130101FE232C8100B1
:104FF000232A91001304050023263101232E1100DA
:105000002328210193840500EFB0CFEC9307200003
:105010008326C405232EF404832784051307100078
:105020009309050093871700232CF4046396E60880
:105030008327840263860700737004306F000000CA
:1050400097B701009387475183A70700639A070822
:105050001309440013050900EFB00FF897B70100DA
:10506000938747510325C40283A7070063F6A7006F
:1050700097B7010023A0A75093054001EF3050459A
:1050800097B701009387C75F930509003385A70091
:10509000EFB04FEC97B701009387474F83A7070006
:1050A0000327C40283A7C70263F8E70063860400EE
:1050B0009307100023A0F400032481018320C10181
:1050C0008324410103290101138509008329C100BB
:1050D000130101026FB08FDF737004306F000000A6
:1050E0009305840117B5010013058568EFB08FE6BD
:1050F0006FF05FFA930705006308050673700430CC
:1051000017B701001307C74683260700639E0602F0
:1051100003A6C70593062000130500006316D600FA
:1051200023AE07041305100083270700638C0700D4
:1051300097B701009387874503A707000327470414
:10514000631C07026780000097B60100938606443F
:1051500003A6060083A6060083264604938616004F
:105160002322D6046FF0DFFA97B701009387074236
:1051700083A707006FF09FF803A7070083A6070027
:10518000832747049387F7FF2322F70483A7460466
:10519000E39A07FA7360043067800000130101FB93
:1051A0002322910423202105232C4103232A510388
:1051B0002328610323267103232611042324810459
:1051C000232E310323248103232291032320A103CF
:1051D00017B901001309893C17BB0100130B4B3BA6
:1051E00097B401009384043B97BA0100938ACA3AAA
:1051F000130A1000930B90008327090003A70700F0
:105200006306071683A7C70083A90700EFD09FCEC8
:10521000EFD0DFCF83270B00130C05006368F50C7C
:1052200097B7010023A6A73613060000637635233F
:1052300003A50400B3858941EFC05FCBEFD01FFF0A
:105240006306051603A5040093060000130600007C
:1052500093058100EFC0CFC9E30005FA83278100E1
:10526000E3C207FE8329010183A749016386070082
:1052700013854900EFB04FD6EFD05FC983270B00ED
:10528000130C05006362F50C8327810017B701003A
:1052900023208731E3E8FBFAB317FA0013F707215D
:1052A0006310072013F7770C6316072A93F707029A
:1052B000E38A07F813850900EF00504F6FF09FF85D
:1052C00083A7C70003A4C70083AC07009309440069
:1052D00013850900EFB04FD0832744021305040063
:1052E000E78007008327C4016386470D83270900F1
:1052F00003A70700E31607FC03A70A0097B60100FF
:1053000023A8862997B6010023A8F62897B701009D
:1053100023A6E728EFD09FF16FF0DFF283A7C70045
:1053200003A4C70003AD0700930C440013850C00D1
:10533000EFB08FCA8327440213050400E7800700FB
:105340008327C401638C470B8327090003A7070049
:10535000E31607FC03A70A0097B6010023AEF62266
:1053600097B7010023ACE7226FF01FF2EFD09FB890
:10537000EFD0DFB983270B00130C0500E368F5F6C7
:1053800083A70A0003A504009309000003A60700F1
:10539000B385894117B70100232C871F13361600E8
:1053A000EFC0DFB4EFD09FE8E31E05E8EFB04F9EFB
:1053B0006FF05FE98327840193850900B387FC00C0
:1053C00063E2FC0883A7040063860702232A010026
:1053D000232C9101232E8100EFF08F9D03A5040063
:1053E000930600001306000093054101EFB00FF68D
:1053F000E31E05EE737004306F0000008327840104
:1054000093850C00B307FD006362FD0883A70400C9
:1054100063860702232A0100232CA101232E810089
:10542000EFF00F9903A50400930600001306000097
:1054300093054101EFB08FF1E31805F0737004306C
:105440006F000000032509002322F40023288400B4
:10545000EFB04FB36FF09FE9EFD05FDD8327090016
:1054600083A7C70003A4C700930C440013850C0056
:10547000EFB08FB68327C401638A470583274402B0
:1054800013050400E78007006FF0DFDB0325090048
:105490002322F40023288400EFB0CFAE6FF0DFEAC0
:1054A0008327C10023ACF9006382070AB387870111
:1054B00023A2F90023A83901938549006362FC08FF
:1054C00003A50A00EFB00FAC6FF0DFD7832784018C
:1054D000232884003387F9002322E400636AEC0464
:1054E000330C3C41636EFC0283A704006386070211
:1054F000232A0100232C3101232E8100EFF04F8B52
:1055000003A5040093060000130600009305410163
:10551000EFB0CFE3E31405F6737004306F000000C2
:1055200003A50A0093850C00EFB0CFA56FF01FF51F
:105530000325090093850C00EFB0CFA46FF01FF492
:1055400003250900EFB00FA46FF0DFCF73700430B4
:105550006F0000008327C10083A6890123A83901B9
:105560003387D70023A2E9006362EC06B307FC404F
:1055700063EAD70683A7490213850900E78007007D
:1055800083A7C901E39047CD83A689018327C10082
:1055900003A70400B387D70063060702232A01008C
:1055A000232CF100232E3101EFF08F8003A504009E
:1055B000930600001306000093054101EFB00FD9D8
:1055C000E31205C8737004306F0000006374FC00C0
:1055D000E372F7FA0325090093854900EFB08F9A2B
:1055E0006FF05FC603A50A0093854900EFB08F995D
:1055F0006FF05FC5130101FF2324810023261100F2
:10560000232291002320210117B40100130484F800
:10561000EFF0CF998327040063840704EFF04F9CD9
:1056200083270400638A0702930800001308000020
:1056300093070000130720009306000013060040A4
:1056400097B50100938585D717050000130545B56B
:10565000EFC01F9E63140506737004306F000000D6
:1056600017B901001309891413050900EFB00F8C55
:1056700097B401009384C41413850400EFB00F8B1A
:10568000130600009305C0001305400097B7010002
:1056900023A627F197B7010023A097F0EFB0CFB66C
:1056A00017B701002328A7EE6306050297B501008E
:1056B000938545D0EFC04FF06FF05FF68320C100B7
:1056C0000324810083244100032901001301010107
:1056D00067800000737004306F000000638A050A61
:1056E000130101FD232A5101930A05001305C0028D
:1056F000232481022322910223202103232E31011E
:10570000232C410123261102232861012326710144
:105710001309070093890600130A06009384050005
:10572000EF00C07013040500630C0502EFF00F8852
:1057300097B70100938707E683A70700638E0704E6
:10574000EFF00F8A1305440023205401232C94000A
:10575000232E44012320340323222403EFA01FFF20
:10576000130504008320C102032481028324410223
:10577000032901028329C101032A8101832A4101EE
:10578000032B0101832BC10013010103678000007B
:10579000737004306F00000097BB0100938B0B0106
:1057A00013850B00EFA09FF817BB0100130B4B01F3
:1057B00013050B00EFA09FF7130600009305C00030
:1057C0001305400097B7010023AA77DD97B70100C2
:1057D00023A467DDEFB04FA317B70100232CA7DA8E
:1057E000630A050097B501009385C5BCEFC0CFDC07
:1057F0006FF01FF5737004306F000000630E050634
:10580000130101FE232C8100232E1100232A910075
:1058100017B40100130404D88328040013080500FA
:105820001305000063800804930407002322B100DD
:10583000138706002324C10023260101930650008C
:1058400063C0B604EFE0DFD693072000630EF504D3
:105850000325040093060000130600009305410091
:10586000EFB0CFAE8320C101032481018324410125
:105870001301010267800000737004306F000000A4
:1058800093054100930600001306070013850800E6
:10589000EFB05FB88320C10103248101832441015B
:1058A0001301010267800000032504009306000035
:1058B0001386040093054100EFB04FA96FF09FFAE3
:1058C000630605000325050067800000737004303F
:1058D0006F00000063160500737004306F00000055
:1058E000130101FF23261100232481001304050066
:1058F000EFE0DFEB032544013334A000EFE05FEE7F
:10590000130504008320C100032481001301010159
:105910006780000063160500737004306F0000009C
:10592000130101FF23248100130405002326110025
:10593000EFE0DFE703240402EFE09FEA8320C100E9
:105940001305040003248100130101016780000096
:1059500063160500737004306F000000130101FF2F
:105960002324810023229100138405009304050061
:1059700023261100EFE09FE323A08402032481008B
:105980008320C10083244100130101016FE05FE522
:10599000130101FF1305C0012324810023261100F8
:1059A000EF00C0481304050063080500232005002C
:1059B00013054500EFA09FD7130504008320C10005
:1059C00003248100130101016780000063020502C6
:1059D000B70700FFB3F7F500638607007370043064
:1059E0006F000000639A0500737004306F000000C0
:1059F000737004306F000000130101FE232C81003E
:105A0000232821012326310123244101232251018E
:105A1000232E1100232A9100930907001389060001
:105A2000930A060013840500130A0500EFE05FB82F
:105A30006318050063860900737004306F0000006E
:105A4000EFD04FCB83240A00B3779400631209048C
:105A50006382070463880A009347F4FFB3F7970053
:105A60002320FA00EFD08FFC8320C10103248101A1
:105A70001385040003290101832441018329C10006
:105A8000032A8100832A410013010102678000007C
:105A9000E302F4FCE38809FCB335500193958501DA
:105AA00063060900B7070004B3E5F5001386090093
:105AB000B3E5850013054A00EFE0CFE1EFD00FF723
:105AC00063140500EFA0DFACEFE01FD6931765006D
:105AD0009309050063DA0700B70400019384F4FF1B
:105AE000B3F499006FF05FF8EFE05FCC83290A0010
:105AF000B377340163100902638A070063880A00E0
:105B00009347F4FFB3F737012320FA00EFE05FCDAE
:105B10006FF09FFCE31CF4FE6FF05FFE630C05006A
:105B2000B70700FFB3F7F500638A0700737004300E
:105B30006F000000737004306F000000130101FF5C
:105B40002324810013040500232611002322910041
:105B50002320210113890500EFE05FC583240400A1
:105B60009345F9FFB3F795002320F400EFE05FC7FA
:105B70008320C10003248100138504000329010050
:105B8000832441001301010167800000130101FF1C
:105B9000232481001304050023261100EFA09FB3E6
:105BA00003240400EFA09FB28320C100130504006A
:105BB000032481001301010167800000630C0500CC
:105BC000370700FFB3F7E500638A070073700430FE
:105BD0006F000000737004306F0000006F30002809
:105BE000B70700FFB377F6006386070073700430D1
:105BF0006F00000063160600737004306F00000031
:105C0000130101FE232C81002328210123263101C9
:105C100023244101232E1100232A91001389060019
:105C200093890500130A050013040600EFE05F984E
:105C3000631E050463060900737004306F000000E2
:105C4000EFD04FAB83240A009385090013050A00A7
:105C5000B3E49900EFF09FF6B3779400630AF40879
:105C600083240A00EFD08FDC8320C101032481014B
:105C70001385040003290101832441018329C10004
:105C8000032A81001301010267800000EFD08FA674
:105C900083240A009385090013050A00B3E4340144
:105CA000EFF0DFF1B3F7840063848704E30A09FAB5
:105CB000B705000513060900B365B40013054A00D3
:105CC000EFE04FC1EFD08FD663140500EFA05F8CDB
:105CD000EFE09FB5931765009304050063D40702B6
:105CE000B70700019387F7FFB3F4F4006FF0DFF715
:105CF00083270A001344F4FFB3F787002320FA0038
:105D00006FF05FF6EFE09FAA83240A00B377940058
:105D1000639887009347F4FFB3F797002320FA00B6
:105D2000EFE01FAC6FF0DFFB130101FF23248100C4
:105D3000232611001304050023229100EFD08F9B2E
:105D40008327440063860702032504019304C400EB
:105D5000631895006F008003032504016308950212
:105D6000B7050002EFE04FE183274400E39607FE0A
:105D700013050400EF008023032481008320C10069
:105D800083244100130101016FD04FCA73700430A6
:105D90006F000000630C0500370700FFB3F7E50054
:105DA000638A0700737004306F0000007370043062
:105DB0006F0000006F30800A630C0500B70700FF1A
:105DC000B3F7F500638A0700737004306F000000BA
:105DD000737004306F000000130101FF2324810061
:105DE000232291002326110013040500938405004B
:105DF000EFE0DF9B0327040093C7F4FFB377F700BE
:105E00002320F400032481008320C1008324410067
:105E1000130101016FE0DF9C630605000325850186
:105E2000678000001305000067800000130101FF78
:105E3000232481002326110013040500EFD08F8B4B
:105E400097A701009387C77583A70700639C070482
:105E5000B797010017B70100130707989387C7FF8B
:105E600097A6010023A4E67417A70100232EF7725A
:105E700017B701002324F79697A70100938787722D
:105E800017B70100232AF7949307100017A7010002
:105E90002320077217A701002326077017A7010008
:105EA0002320F77063120402EFD04FB8EF10C058F0
:105EB00013040000130504008320C10003248100A3
:105EC00013010101678000001305840093773500FA
:105ED0006398070CB79701001307F5FF9387A7FF97
:105EE000E3E4E7FC97A601009386466C83A70600CF
:105EF0006F00400103A70700630A070093860700AD
:105F00009307070003A74700E366A7FE17A7010052
:105F100013074769E38AE7F803A7070013060001A0
:105F20001384870023A0E60003A74700B306A74019
:105F3000637ED6023388A7002322D80023A2A700BD
:105F40008325480097A60100938646666F0080006F
:105F50009306070003A7060003264700E36AB6FE80
:105F60002320E80023A0060103A7470097A701000C
:105F70009387076783A70700B387E74017A7010048
:105F80002320F766EFD08FAAE30204F21305040082
:105F90008320C100032481001301010167800000F8
:105FA0001375C5FF130545006FF0DFF263080506A2
:105FB000130101FF2324810023261100130405008F
:105FC000EFC05FF3930584FF0326C4FF17A701000A
:105FD0001307C75D6F008000138707008327070042
:105FE00083A64700E3EAC6FE232CF4FE2320B70075
:105FF00097A701009387C75E03A707008327C4FF05
:10600000032481008320C100B387E70017A70100A4
:106010002328F75C130101016FD04FA167800000B6
:1060200097A701009387C75B03A50700678000005F
:10603000678000003367B5001377370093070500CA
:10604000631207049308D6FFB30815011307050070
:10605000938605006378150303A80600130747001D
:1060600093864600232E07FFE36817FF9347F5FF4B
:10607000B387170193F7C7FF93874700B385F500F0
:10608000B307F5003306C50063F4C70C93864500DB
:1060900013884700B3B6D70033B8050133E7F500DE
:1060A00093C616001348180013773700B3E60601AD
:1060B000133717003377D700330EF6409386170057
:1060C000630807061337AE006314070613532E0048
:1060D0001388050093860700130700008328080033
:1060E000130717001308480023A0160193864600E3
:1060F000E36667FE1377CEFFB385E500B387E7005D
:106100006306EE0483C60500138717002380D700BB
:10611000637EC70283C6150013872700A380D700BC
:106120006376C70203C725002381E700678000006C
:10613000B307F640B387F5009385150003C7F5FF55
:1061400093861600238FE6FEE398F5FE6780000035
:1061500067800000B367C50093F73700B308C50038
:106160006382070E63761511B307A04093F73700DB
:10617000138737009306500093F5F50F13081500A9
:106180003383A8401306F6FF6374D700130750004B
:106190006368E60E6380070E2300B5001307100046
:1061A000638EE700A300B500130730001308250035
:1061B0006396E700130835002301B50013968500A8
:1061C00033E6C500139705013367E6003303F34058
:1061D00093968501B366D70013562300B307F500E5
:1061E0001307000023A0D700130717009387470069
:1061F000E36AC7FE1377C3FFB307E8006300E30851
:106200002380B70013871700637C1703A380B700B0
:1062100013872700637617032381B700138737009E
:1062200063701703A381B70013874700637A1701D0
:106230002382B7001387570063741701A382B70046
:106240006780000093F5F50F13978500B365B700DD
:10625000139705013367B700E37415FF9307050033
:106260009387470023AEE7FEE3EC17FF678000004B
:1062700067800000130805006FF05FF4678000007E
:10628000930705006FF0DFF783470500130705004C
:10629000638C07001305150083470500E39C07FE88
:1062A0003305E540678000001305000067800000AB
:1062B000130515008347F5FF9385150003C7F5FF08
:1062C00063880700E386E7FE3385E74067800000C8
:1062D000930700006FF05FFF93070500938515009B
:1062E00003C7F5FF93871700A38FE7FEE31807FEA8
:1062F0006780000083460500930700026398F6005C
:106300001305150083460500E38CF6FE938756FDC2
:1063100093F7D70F638007049307050093050000E8
:10632000638806041305000093871700138606FD93
:106330001317250083C607003305A70013151500A2
:106340003305A600E39206FE638405003305A040F2
:1063500067800000938536FD8346150093B51500D0
:1063600093071500E39006FC130500006FF0DFFDB6
:10637000130500006780000083A705002380A700A5
:1063800083A705009387170023A0F500678000000E
:1063900097A601009386062283A7060017370300FD
:1063A0001307474613861700B307F7002380A7009B
:1063B00097A5010023A0C5209307A000630AF5005C
:1063C000930700046308F6001305000067800000CF
:1063D000E30C06FE370610F0130717008347F7FF9C
:1063E0002320F6F083A706009387F7FF97A5010007
:1063F00023A2F51CE39207FE13050000678000004E
:10640000130101EB2322911423202115232A511378
:10641000232481132326111423248114232E3113C2
:10642000232C411323286113232671132322911354
:106430002320A113232EB111930405001389050015
:106440002326C100130C5002930A900083470900D1
:1064500063888703638C070603A404006F00800031
:10646000638607062300F40003A40400130919003F
:106470001304140023A0840083470900E39287FFDC
:10648000034619009308190093860800130D0002B3
:106490009309F0FF130AF0FF1308000013055005DD
:1064A0009307D6FD93F7F70F13891600636EF53A3D
:1064B00017A70100130707B593972700B387E700D5
:1064C00083A70700B387E700678007008320C11414
:1064D0000324811483244114032901148329C11343
:1064E000032A8113832A4113032B0113832BC11227
:1064F000032C8112832C4112032D0112832DC11113
:106500001301011567800000930C80002324010013
:106510009307100063DA071D8327C10003A404005A
:10652000938B770093F68BFF03AB060083A946009D
:10653000938786002326F10013860C009306000043
:1065400013050B0093850900EF2080282328A10064
:106550009307000063803733930D4101930B1000C4
:1065600013860C009306000013050B0093850900A9
:10657000EF1050489306000013860C00130B050023
:1065800093890500EF20C0248327810023A0AD005C
:1065900093861B00938D4D0063863701938B060015
:1065A0006FF01FFCE37C9BFF63D24603930704005C
:1065B0002380A70103A40400130AFAFF9307140021
:1065C00023A0F40013840700E3C446FF93962B0036
:1065D00093070101B386D7006F0080029387770588
:1065E0002300F40003A40400938BFBFF93871B009C
:1065F0001304140023A084009386C6FFE358F0E43C
:1066000083A70600E3ECFAFC938707036FF05FFDB6
:1066100083A70400930600030327C1002380D7004B
:1066200083A7040093064700930C0001138617000C
:1066300023A0C40013068007A380C70003A404009E
:1066400023240100930707001304140023A08400EF
:1066500003AB0700930900002326D1006FF0DFEDA4
:106660008327C10083AC0700938B470063880C2805
:10667000635C40259307D002631EFD2083C70C0096
:106680006388070263D8092483A60400938C1C0046
:10669000130AFAFF2380F60003A404001304140075
:1066A00023A0840083C70C00E39E07FC63524003D1
:1066B00003A40400930700022300F40003A40400D1
:1066C000130AFAFF1304140023A08400E3160AFE41
:1066D000232671016FF09FD7232401009307100038
:1066E000930CA000E3CA07E38327C10003A40400BE
:1066F000938647006FF0DFF503C616009306090086
:106700006FF01FDA83A70400930650022380D7009E
:1067100003A404001304140023A084006FF01FD30B
:10672000930C0001232401006FF09FDE8327C1003A
:1067300003C616009306090083A907009387470044
:106740002326F100E35E0AD4138A09009309F0FFBF
:106750006FF01FD503C61600130DD0029306090073
:106760006FF01FD49347FAFF93D7F74103C6160083
:10677000337AFA00930609006FF09FD203C6160021
:10678000130D0003930609006FF09FD183C5160017
:10679000930906FD93060900938705FD13860500FE
:1067A000E3E2FAFA93972900B3893701938616003A
:1067B00093991900B389B90083C50600938909FD2F
:1067C000938705FD13860500E3FEFAFC6FF09FF743
:1067D0000327C10083A7040083260700130747008F
:1067E0002326E1002380D70003A40400130414002F
:1067F00023A084006FF09FC59307100063D4070F98
:106800008327C1009386770093F686FF93878600DF
:106810002326F10083A9460083A7060063DE090E44
:1068200083A604001306D002B307F0402380C600FD
:1068300003A40400B336F000B3093041130414007C
:1068400023A08400138B0700B389D940930CA000C8
:10685000232401006FF05FCE03C616001308180052
:10686000930609006FF0DFC383A7040013890800B3
:106870006FF09FE9E3729BCF93071000930B00002A
:1068800093061000E3C447D36FF05FD497AC0100C8
:10689000938C4CB39385090013850C00EF10C03D19
:1068A000330AAA406352400303A404002300A40156
:1068B00003A40400130AFAFF1304140023A08400A5
:1068C000E3160AFE130A000083C70C00E38207E008
:1068D000E3CC09DA9389F9FF1307F0FFE396E9DACD
:1068E0006FF0DFDC8327C1009386470083A7070092
:1068F0002326D10093D9F7416FF05FF26356400130
:106900009307D002E314FDF897AC0100938C8CAB95
:10691000930780026FF01FD7138B0700930CA00022
:106920002324010003A404006FF01FC1130101EB35
:10693000232E3113B70900409387F9FF23248114D4
:1069400023229114232C4113232A5113232611149B
:106950002320211523286113232671132324811357
:10696000232291132320A113232EB111130A050012
:106970002324B10017A401001304C4C3973A0300F1
:10698000938A4AE8979401009384447D2326F1007A
:10699000930550021305A00013080004B70610F079
:1069A00083470A00638EB7046388070A032704003D
:1069B000130A1A00130617003387EA0097A801008C
:1069C00023AAC8BE2300F7006380A708E31A06FDC8
:1069D00017370300130707E3130717008347F7FF71
:1069E00023A0F6F0832704009387F7FF17A6010082
:1069F0002322F6BCE39207FE83470A00E396B7FA28
:106A000083461A0013051A0013070500930B0002B2
:106A1000130BF0FF130CF0FF130800009305500553
:106A2000930890009387D6FD93F7F70F130A17008A
:106A300063ECF54493972700B387970083A707007B
:106A4000B38797006780070017370300130787DBBA
:106A5000E31406F86FF0DFF48320C11403248114DB
:106A600083244114032901148329C113032A8113A8
:106A7000832A4113032B0113832BC112032C811290
:106A8000832C4112032D0112832DC1111301011515
:106A900067800000930C8000130D00009307100026
:106AA00063DA0721832781009387770093F787FFB5
:106AB00083AD070003AB4700138787002324E10061
:106AC00013860C009306000013850D0093050B0040
:106AD000EF1010502328A10063086D4513094101F0
:106AE0009309100013860C009306000013850D0017
:106AF00093050B00EF10007013860C009306000046
:106B0000930D0500138B0500EF10904C2320A90076
:106B10009389190013094900E3166DFDE3F49DFD07
:106B200013060004B70610F063D48903832704001A
:106B300013871700B387FA0097A5010023ACE5A6D9
:106B400023807701630AC706130CFCFFE3C089FFAB
:106B50008327C1001305C10093089000B386F90094
:106B60009396260093070101B386D7001308A0006F
:106B700013030004370610F0E38CA6E083A7060099
:106B80009305000363F4F8009305700503270400E0
:106B9000B387B700930517003387EA0017AE0100EB
:106BA000232ABEA02300F70063860737638C653273
:106BB0009386C6FF6FF05FFC17370300130787C487
:106BC000130717008347F7FF23A0F6F0832704007D
:106BD0009387F7FF97A5010023AEF59CE39207FE8C
:106BE000130CFCFF6FF09FF68327040013060004CC
:106BF0001387170097A5010023AEE59AB386FA0024
:106C0000930500032380B6006308C75093872700CD
:106C100097A6010023A0F69A3387EA00930680071F
:106C20002300D700173703001307C7BDB70610F0BE
:106C30006392C702130717008347F7FF23A0F6F0FC
:106C4000832704009387F7FF17A601002324F696F5
:106C5000E39207FE83278100930C0001130D0000CF
:106C60009387470003278100130B0000832D070043
:106C70002324F1006FF0DFE48327810083AC070059
:106C800013894700638E0C4C6358802B9307D00206
:106C90006394FB3E03C70C00930507006314072AA7
:106CA0006F00002F93071000930CA000130D00003D
:106CB000E3CA07DF83278100938747006FF09FFABD
:106CC000832781008346170013070A0003AB0700E0
:106CD000938747002324F100E3560CD4130C0B00D8
:106CE000130BF0FF6FF01FD483461700930BD002F5
:106CF00013070A006FF01FD39347FCFF93D7F741A8
:106D000083461700337CFC0013070A006FF09FD105
:106D100083461700930B000313070A006FF09FD000
:106D200003461700138B06FD13070A00930706FDA1
:106D300093060600E3E2F8FA93172B00B387670186
:106D40001307170093971700B387C7000346070080
:106D5000138B07FD930706FD93060600E3FEF8FC80
:106D60006FF09FF783258100832704001306A0009E
:106D700003A7050093861700B387FA0017A5010043
:106D8000232AD5822380E700138945006300C73694
:106D9000930700046384F62A232421016FF05FBF68
:106DA0009307100063DE0735832781001387770080
:106DB000137787FF930787002324F100032B4700F5
:106DC0008327070063560B3E0327040013060004C5
:106DD000930617009795010023AED57C3387EA0010
:106DE0009305D0022300B700638CC638B307F04088
:106DF0003337F000330B6041938D0700330BEB40CA
:106E0000930CA000130D00006FF09FCB834617007A
:106E10001308180013070A006FF0DFC0834617003D
:106E200013070A006FF01FC08327040093060004B5
:106E30001387170017960100232EE676B387FA0012
:106E4000130650022380C700E314D7B4173703009A
:106E50001307479BB70610F0130717008347F7FF88
:106E600023A0F6F0832704009387F7FF179601000D
:106E70002322F674E39207FE6FF09FB1930C00019A
:106E8000130D00006FF09FC18327040093060004D8
:106E9000130A05001387170017960100232CE670CC
:106EA000B387FA00130650022380C700E312D7AE5F
:106EB0001737030013070795B70610F013071700DD
:106EC0008347F7FF23A0F6F0832704009387F7FF9B
:106ED000179601002320F66EE39207FE130A0500C1
:106EE0006FF01FAB173703001307C7911307170085
:106EF0008347F7FF2320F6F0832704009387F7FFEB
:106F00009795010023A8F56AE39207FE9386C6FFD2
:106F10006FF09FC6173703001307C78EE39805FC71
:106F20009386C6FF6FF05FC5E3FA9DBB930910001F
:106F30006FF01FBF130C000003C70C009305070080
:106F4000E30C07E49308F0FF1305A0001308000406
:106F5000B70610F0635E0B0C83270400138617003E
:106F6000B387FA00179301002326C3642380E70048
:106F70006382A5086308060B938C1C0003C70C00F2
:106F8000130CFCFF93050700E31607FCE35680E1B2
:106F9000832704009305000213060004B70610F0CF
:106FA0006F00C000130CFCFFE3080CDE1387170012
:106FB000B387FA002380B70017950100232CE55E04
:106FC00093070700E310C7FE1737030013078783F3
:106FD000130717008347F7FF23A0F6F08327040069
:106FE0009387F7FF179501002326F55CE39207FED0
:106FF0006FF05FFB173703001307C780E30E06F639
:10700000130717008347F7FF23A0F6F08327040038
:107010009387F7FF17960100232EF658E39207FE99
:107020006FF09FF5172703001307C77D6FF05FFD13
:10703000130BFBFFE3121BF36FF05FF51727030041
:107040001307477CB70610F0130717008347F7FFB5
:1070500023A0F6F0832704009387F7FF179601001B
:10706000232AF654E39207FE232421016FF05F9256
:10707000979C0100938C0C3593050B0013850C0035
:10708000EF00903F330CAC40E35880EB83270400C3
:1070900013060004B70610F06F00C000130CFCFFCD
:1070A000E30A0CE813871700B387FA0023807701FF
:1070B0009795010023A0E55093070700E310C7FE52
:1070C0001727030013070774130717008347F7FFF9
:1070D00023A0F6F0832704009387F7FF979501001C
:1070E00023AAF54CE39207FE6FF05FFB172703001E
:1070F00013074771E39806F4232421016FF05F8999
:10710000832781001387470083A707002324E1001A
:1071100013DBF7416FF01FCB172703001307876EB0
:10712000B70610F0130717008347F7FF23A0F6F008
:10713000832704009387F7FF17960100232CF64658
:10714000E39207FE93071000179701002324F746E8
:1071500093078007172703002306F76A6FF09FAF96
:10716000635680019307D002E394FBF0979C0100E3
:10717000938C4C2513078002930580026FF09FDCEF
:107180009726030093860668370610F0938616004C
:1071900003C7F6FF2320E6F0032704001307F7FFD9
:1071A0009795010023A8E540E31207FE6FF01FC486
:1071B000938D0700930CA000130D00006FF05F90FB
:1071C000B70710F023A0A7F26F000000130101FC25
:1071D000130341022322B10293050300232E110061
:1071E0002324C1022326D1022328E102232AF1020B
:1071F000232C0103232E110323266100EFF00FF34C
:107200008320C10113050000130101046780000001
:10721000130101FB13038103232481022326A10010
:10722000232CC10213040500130603001305C1003B
:10723000232611022322F104232ED1022320E1046C
:107240002324010523261105232E6100EFF04F9B17
:107250008327C100238007000325C1008320C102CA
:107260003305854003248102130101056780000076
:10727000B70710F083A647F403A607F403A747F463
:10728000E31AD7FEB7260000938606F4B306D600AD
:1072900033B6C600B305E60023A4D7F423A6B7F49B
:1072A00067800000B70710F003A747F403A607F4B0
:1072B00083A647F4E31AD7FEB7260000938606F4A8
:1072C000B306D60033B6C60023A4D7F4B305E60050
:1072D00023A6B7F49307000873A047306780000027
:1072E000130101FF23248100232611009797010039
:1072F0009387C72C179401001304042C03A70700DD
:10730000832704001306F07C9306470693874706FD
:107310009795010023A4D52A9795010023AEF5285F
:10732000634AD6008320C1000324810013010101B8
:1073300067800000130747899797010023A0E7287B
:10734000EF00D009930710006316F502032704002D
:10735000B71700009387F77613050000E3D4E7FC26
:10736000EFF01FE6032481008320C1001301010117
:107370006FB05FB71795010013054505EFF01FE5E6
:1073800013052000EFF0DFE3032481008320C10018
:10739000130101016FB01FB5179501001305C50456
:1073A0006FF0DFE217950100130585046FF01FE20F
:1073B000130101FF232481002322910023261100C1
:1073C000B714000017940100130404039387843852
:1073D000130000009387F7FFE39C07FE13050400EA
:1073E000EFF0DFDE6FF09FFE130500006F00C06D51
:1073F000130101FF23261100EF00407E1307100048
:1074000093070000631AE5008320C100138507007D
:10741000130101016780000017950100130505FBAA
:10742000EFF0DFDA8320C100930720001385070007
:107430001301010167800000737004306F000000C9
:1074400067800000737004306F000000130101FFBB
:1074500023248100232611001794010013044417EC
:1074600013050000EFC0DF93832704009387170004
:1074700017970100232EF7146FF09FFE130101FFF1
:107480002324810023229100232611009304050068
:107490001304100013050000EFC09F909306000036
:1074A0001306F0FF9305000013850400EF90DFDA68
:1074B0009306000013060000930500006302850296
:1074C000138504009797010023AA8710EF90DFB976
:1074D000E30285FC9797010023A287106FF09FFBC2
:1074E00093060000130600009305000013850400B6
:1074F000EF909FB7E30085FA9797010023A0870ECE
:107500006FF05FF9130101FE232C8100232A910003
:107510002328210123263101232441012322510163
:1075200023206101232E110093090500179B010000
:10753000130BCB09979A0100938A0A091799010046
:1075400013090909179A0100130ACA081304100045
:10755000930430009306000013060000930500001A
:1075600013850900EF905FCF6306850097970100B0
:1075700023A68706130500009797010023AA070496
:10758000EFB08F9A630605009797010023A8870440
:1075900003250B00EFB08FC013050000EFB0CF98AC
:1075A000630695009797010023AA87021305000040
:1075B00093051000EFB04FA413050000EFB0CF9675
:1075C000630695009797010023AA870003A50A0088
:1075D000EFB0CFBC832709006386070097970100AF
:1075E00023AE87FE930600001306000093050000FB
:1075F00013850900EF905FA7630685009797010048
:1076000023AE87FC832709006386870097970100D4
:1076100023A687FC13050000EFB00F9163068500D9
:107620009797010023AC87FA93050000130500002B
:10763000EFB08F9C83270A009387170017970100EC
:10764000232AF7F86FF01FF1130101FC23244103F3
:10765000179A0100130A4AF8232C8102232A910267
:1076600023282103232631032322510323206103EE
:10767000232E7101232E1102232C810113040500F6
:10768000930B0A00130B200093044000930A500050
:107690001309B00093096000930610001306000060
:1076A00093850B0013050400EF901F9C1305040045
:1076B000EFA00FD8930710006306F500179701009D
:1076C000232EF7F0930600001306000093058100B7
:1076D00013050400EF905FB8930710006306F500F0
:1076E00017970100232CF7EE03270A008327810058
:1076F0006308F70093071000179701002320F7EEA7
:1077000013050400EFA0CFD2630805009307100013
:10771000179701002324F7EC9306000013060000DE
:1077200093850B0013050400EF901F9413050400CC
:10773000EFA00FD0930710006306F5001797010024
:10774000232EF7E89306000013060000930581003E
:1077500013050400EF905FB0930710006306F50077
:1077600017970100232CF7E613050400EFA04FCC78
:107770006308050093071000179701002320F7E620
:1077800003270A00832781006308F700930710008E
:10779000179701002324F7E42324610193060000D6
:1077A000130600009305810013050400EF90DF8BA2
:1077B00083278100938717002324F100E3F0F4FE70
:1077C00013050400EFA0CFC6930730006308F5004F
:1077D00093071000179701002322F7E0930610008B
:1077E0001306000093058100130C1000130504001C
:1077F00023248101EF905F87930610001306000099
:10780000930581001305040023240100EF90DF8518
:1078100013050400EFA0CFC163065501979701003F
:1078200023AE87DB9306100013060000930581004A
:1078300013050400EF905F836308050093071000B1
:1078400017970100232CF7D89306000013060000B9
:107850009305810013050400EF901F816308050064
:107860009307100017970100232AF7D6232401005D
:1078700093061000130600009305C10013050400D1
:10788000EF909F9D930710009306000013060000E1
:107890009305C1006306F500179701002320F7D474
:1078A0008327C100032881001305040013C7F7FFD5
:1078B0006308F80093071000179801002320F8D2FE
:1078C0002326E100EF905F99930710006306F5000F
:1078D000179701002324F7D0832781008326C10056
:1078E00013871700638AD71C93071000979601002F
:1078F00023A6F6CE2324E100E3FCE4F613050400FE
:10790000EFA00FB36308050093071000179701005D
:107910002326F7CC9307A00093060000130600006F
:1079200093058100130504002324F100EF90CFF3A9
:10793000930710006306F500179701002320F7CA8C
:107940009306000013060000930581001305040050
:1079500023242101EF904FF1930710006306F500F7
:1079600017970100232CF7C613050400EFA04FACB6
:107970006308650193071000179701002320F7C6DD
:10798000930790002324F1009306100013060000D3
:107990009305810013050400EF900FED930710008D
:1079A0006302F51017970100232AF7C2832781008D
:1079B0009387F7FF2324F100E3E8F9FC13050400A3
:1079C000EFA00FA763085501930710001797010058
:1079D0002326F7C0930610001306000093058100CC
:1079E00013050400EF904FE86308050093071000AB
:1079F000179701002324F7BE93060000130600002A
:107A00009305810013050400EF900FE6630805005D
:107A100093071000179701002322F7BC930770000B
:107A20002324F100130C100093060000130600003D
:107A30009305C10013050400EF901F8263068501C2
:107A40009797010023AC87B9832781008326C10063
:107A5000138717006380D7049797010023A087B985
:107A60002324E100E372E9FC13050400EFA04F9C1E
:107A70006308050093071000179701002320F7B64D
:107A800083270A0093871700179701002326F7B46E
:107A90006FF09FC0938717002324F100E376F9F875
:107AA0006FF09FFC832781009387F7FF2324F10069
:107AB000E3ECF9EC6FF09FF0938717002324F100BB
:107AC000E3F8F4DA6FF09FE3130101FF2322910042
:107AD00013060000930405009305400013055000B1
:107AE0002326110023248100EF801FF297950100C7
:107AF0009385C59113040500EFA00FAC1387040014
:107B00009306040093080000130800009307000088
:107B10001306004097950100938585901705000096
:107B20001305C5B2EFA0CFD013051000EF900FC31F
:107B3000979501009385458F13040500EFA0CFA70B
:107B40009306040093080000130800009307000048
:107B50001307000013060040979501009385858D5B
:107B6000170500001305459AEFA08FCC930800007D
:107B70001308000097970100938707A513072000BB
:107B80009306000013060040979501009385058B2E
:107B9000170500001305C58BEFA08FC993060400DD
:107BA000032481008320C100832441009308000046
:107BB0001308000097970100938747A1130730002F
:107BC00013060040979501009385C58717050000AF
:107BD0001305058B130101016FA08FC517970100D5
:107BE0001307879F979601009386C69D83270700FA
:107BF00083A606006398F60093071000979601008D
:107C000023AEF69C979701009387C79C17960100B7
:107C10001306069B83A60700032606006308D60208
:107C2000979601009386869B0327070003A506000D
:107C300083A707009796010023A6E6981335150041
:107C400017970100232EF79667800000032707008F
:107C500083A7070093061000179601002320D698EB
:107C6000130500009796010023AEE69417970100D4
:107C70002328F79467800000B305B500930705003B
:107C80006386B70003C70700631607003385A74064
:107C900067800000938717006FF09FFE130101FBC0
:107CA00023229104232C4103232291032326110430
:107CB0002324810423202105232E3103232A510369
:107CC0002328610323267103232481032320A10396
:107CD000232EB101930C0500138A050093040000C4
:107CE00063DE05003305A0403337A000B305B04084
:107CF000930C0500338AE5409304F0FF63DA060035
:107D00003306C040B337C000B306D040B386F64058
:107D1000930A06009389060013840C0013090A00D5
:107D200063960628178B0100130BCB586370CA1695
:107D3000B70701006372F6149307F00F63F4C700EE
:107D400093098000B3573601330BFB0083470B00C8
:107D500013050002B3873701B309F540638C0900AE
:107D6000B3153A01B3D7FC00B31A360133E9B700B3
:107D700033943C0113DB0A0193050B001305090042
:107D8000EF00507C130A050093050B00939B0A013A
:107D900013050900EF00907693DB0B0193050500B6
:107DA00013850B00EF00D072131A0A0193570401D8
:107DB000B367FA0063FAA700B387570163E6570178
:107DC00063F4A700B38757013389A74093050B00DD
:107DD00013050900EF001077130A050093050B0047
:107DE00013050900EF0090711314040193050500B9
:107DF000131A0A0113850B0013540401EF00506D90
:107E000033648A00637AA400330454016366540126
:107E10006374A400330454013304A4403354340184
:107E200093050000638A040033048040B337800068
:107E3000B305B040B385F540130504008320C104A9
:107E40000324810483244104032901048329C103F9
:107E5000032A8103832A4103032B0103832BC102DD
:107E6000032C8102832C4102032D0102832DC101C9
:107E70001301010567800000B707000193090001A5
:107E8000E362F6EC930980016FF0DFEB631A060002
:107E90009305000013051000EF005066930A0500DB
:107EA000B707010063FAFA0E9307F00F63F4570166
:107EB00093098000B3D73A01330BFB0083470B00D3
:107EC0001305000233095A41B3873701B309F5405E
:107ED000E38209EAB39A3A01335BFA00B3153A0137
:107EE000B3D7FC0093DB0A0133E9B70013050B009D
:107EF00093850B00EF001065130A050093850B00B6
:107F0000139C0A0113050B00EF00505F135C0C017A
:107F10009305050013050C00EF00905B131A0A018E
:107F200093570901B367FA0033943C0163FAA70041
:107F3000B387570163E6570163F4A700B38757017E
:107F4000338BA74093850B0013050B00EF00905F68
:107F5000130A050093850B0013050B00EF00105A60
:107F60009305050013050C00EF00905693160901C8
:107F7000131A0A0193D60601B366DA0063FAA60063
:107F8000B386560163E6560163F4A600B386560134
:107F90003389A6406FF01FDEB70700019309000187
:107FA000E3EAFAF0930980016FF0DFF06376DA001C
:107FB00093050A006FF01FE7B707010063FAF604A4
:107FC000930BF00F33B5DB001315350033D7A60044
:107FD000978701009387072EB387E70083CB0700BD
:107FE00093050002B38BAB00338B7541631C0B020E
:107FF00063E4460163EACC003384CC40B306DA4044
:1080000033B98C0033892641930509006FF09FE155
:10801000B707000113050001E3EAF6FA1305800132
:108020006FF0DFFAB3966601335D7601336DDD00E4
:10803000B35D7A01B3156A0133DC7C0113540D0181
:10804000336CBC0013850D0093050400B319660161
:10805000EF00504F930A05009305040013850D00AF
:1080600033996C01931C0D01EF00504993DC0C0116
:10807000130A05009305050013850C00EF00504519
:10808000939A0A0113570C0133E7EA00930D0A0093
:10809000637EA7003307A701930DFAFF6368A7016A
:1080A0006376A700930DEAFF3307A701330AA740C1
:1080B0009305040013050A00EF00D048930504005F
:1080C000930A050013050A00EF00504393050500CD
:1080D0001304050013850C00EF00903F93150C016D
:1080E000939A0A0193D50501B3E5BA00130704007A
:1080F00063FEA500B385A5011307F4FF63E8A5019E
:1081000063F6A5001307E4FFB385A501939D0D0158
:10811000B70C0100B3EDED001384FCFFB3F78D0045
:1081200033F48900338AA5401385070093050400C2
:108130002326F10093DD0D01EF0090399305040033
:10814000930A050013850D00EF00903813DC090138
:1081500093050C002324A10013850D00EF00503778
:108160008327C10013040C0093050400130C0500C1
:1081700013850700EF00D0358326810013D70A014D
:108180003305D5003307A7006374D700330C9C0177
:10819000B70701009387F7FF935507013377F7007F
:1081A00013170701B3F7FA00B3858501B307F7008A
:1081B0006366BA00631EBA00637CF90033863741F8
:1081C000B3B7C700B385A541B385F5409307060053
:1081D000B307F9403339F900B305BA40B3852541F7
:1081E00033947501B3D767013364F400B3D56501E7
:1081F0006FF05FC3130101FD23229102232A510175
:10820000232611022324810223202103232E31015E
:10821000232C41012328610123267101232481019C
:10822000232291012320A101930A050093840500D4
:10823000639E0638130406009309050017890100A0
:108240001309490763F8C512B7070100138B05002E
:108250006378F6101307F00F3337C7001317370092
:10826000B357E6003309F900834609003387E60077
:1082700093060002B386E640638C0600B394D400F4
:1082800033D7EA003314D600336B9700B399DA0082
:10829000935A040193850A0013050B00EF00902AFE
:1082A0001309050093850A00931B040113050B00B5
:1082B000EF00D02493DB0B01930405009305050028
:1082C00013850B00EF00D0201319090193D7090182
:1082D000B367F900138A040063FEA700B387870021
:1082E000138AF4FF63E8870063F6A700138AE4FFAC
:1082F000B3878700B384A74093850A0013850400E1
:10830000EF0050241309050093850A00138504002B
:10831000EF00D01E93990901930405009305050011
:108320001319090113850B0093D90901EF00501AA5
:10833000B36939011386040063FCA900B309340151
:108340001386F4FF63E6890063F4A9001386E4FF53
:1083500013140A013364C400130A00006F000013F1
:10836000B707000113070001E36CF6EE1307800165
:108370006FF01FEF138A0600631A060093050000D2
:1083800013051000EF00901713040500B707010054
:10839000637EF4129307F00F63F48700130A8000E2
:1083A000B35744013309F90003470900930600025B
:1083B00033074701B386E64063940612B3848440D2
:1083C000130A1000135B040193050B0013850400CE
:1083D000EF0050171309050093050B0013850400E7
:1083E000931B0401EF00901193DB0B019304050034
:1083F0009305050013850B00EF00900D131909017B
:1084000093D70901B367F900938A040063FEA700BC
:10841000B3878700938AF4FF63E8870063F6A700B9
:10842000938AE4FFB3878700B384A74093050B00CA
:1084300013850400EF0010111309050093050B00CC
:1084400013850400EF00900B939909019304050034
:10845000930505001319090113850B0093D9090130
:10846000EF001007B36939011386040063FCA9000B
:10847000B30934011386F4FF63E6890063F4A900AD
:108480001386E4FF13940A013364C4001305040047
:1084900093050A008320C102032481028324410240
:1084A000032901028329C101032A8101832A410191
:1084B000032B0101832BC100032C8100832C41007D
:1084C000032D01001301010367800000B7070001BD
:1084D000130A0001E366F4EC130A80016FF05FEC0D
:1084E0003314D40033DAE400B399DA0033D7EA0066
:1084F000935A0401B394D40093850A0013050A002B
:10850000336B9700EF0010041309050093850A00F0
:1085100013050A00931B0401EF00407E93DB0B015F
:10852000930405009305050013850B00EF00407AC6
:108530001319090113570B013367E900138A04006B
:10854000637EA70033078700138AF4FF6368870000
:108550006376A700138AE4FF33078700B304A740BC
:1085600093850A0013850400EF00C07D1309050000
:1085700093850A0013850400EF00407893040500FA
:108580009305050013850B00EF00807413170B0192
:108590001357070113190901B367E9001387040092
:1085A00063FEA700B38787001387F4FF63E88700A3
:1085B00063F6A7001387E4FFB3878700131A0A0145
:1085C000B384A740336AEA006FF0DFDF63ECD51EA7
:1085D000B707010063F4F6041307F00FB335D700B3
:1085E0009395350033D7B60097870100938787CCE2
:1085F000B387E70003C70700130A00023307B70079
:10860000330AEA4063160A0213041000E3E096E816
:1086100033B6CA00134416006FF05FE7B7070001D6
:1086200093050001E3E0F6FC930580016FF09FFBEA
:10863000B35CE600B3964601B3ECDC0033D4E4004F
:1086400093DB0C01B397440133D7EA0093850B0009
:1086500013050400336BF700B3194601EF00806E79
:108660001309050093850B0013050400139C0C01EE
:10867000EF00C068135C0C0193040500930505002E
:1086800013050C00EF00C0641319090113570B0107
:108690003367E90013840400637EA7003307970162
:1086A0001384F4FF636897016376A7001384E4FFE3
:1086B00033079701B304A74093850B00138504008B
:1086C000EF0040681309050093850B001385040033
:1086D000EF00C062930405009305050013050C002C
:1086E000EF00005F93170B011319090193D70701DE
:1086F000B367F9001386040063FEA700B3879701F0
:108700001386F4FF63E8970163F6A7001386E4FF7E
:10871000B387970113140401B70B01003364C4003D
:108720001389FBFF337D240133F92901B384A7406A
:108730009305090013050D00EF008059935C0401B7
:1087400093050900130B050013850C00EF0040583A
:1087500093D90901130C05009385090013850C00BA
:10876000EF000057130905009385090013050D005C
:10877000EF0000563305850193570B013385A700A1
:10878000637485013309790193570501B387270184
:1087900063E6F402E392F4BCB70701009387F7FFA6
:1087A0003375F50013150501337BFB0033964A0141
:1087B00033056501130A0000E37AA6CC1304F4FF25
:1087C0006FF09FB9130A0000130400006FF01FCC74
:1087D000130101FB2324810423229104232E31035E
:1087E000232291032326110423202105232C410356
:1087F000232A5103232861032326710323248103A1
:108800002320A103232EB101930C050093890500B9
:108810001304050093840500639E062613090600D1
:10882000138A0600978A0100938ACAA863F4C514C4
:10883000B70701006376F6129307F00F63F4C700E1
:10884000130A8000B3574601B38AFA0003C70A002F
:108850001305000233074701330AE540630C0A00A1
:10886000B395490133D7EC0033194601B364B7001F
:1088700033944C01935A090193850A00138504002F
:10888000EF00404C9309050093850A00131B090172
:1088900013850400EF008046135B0B019305050070
:1088A00013050B00EF00C04293990901935704018F
:1088B000B3E7F90063FAA700B387270163E627014E
:1088C00063F4A700B3872701B384A74093850A0008
:1088D00013850400EF0000479309050093850A0003
:1088E00013850400EF008041131404019305050073
:1088F0009399090113050B0013540401EF00403D47
:1089000033E48900637AA4003304240163662401FC
:108910006374A400330424013304A4403355440198
:10892000930500008320C1040324810483244104AF
:10893000032901048329C103032A8103832A4103F4
:10894000032B0103832BC102032C8102832C4102E0
:10895000032D0102832DC101130101056780000071
:10896000B7070001130A0001E36EF6EC130A800159
:108970006FF05FED631A0600930500001305100009
:10898000EF00C03713090500B7070100637AF90E3D
:108990009307F00F63F42701130A8000B3574901CE
:1089A000B38AFA0003C70A0013050002B384294101
:1089B00033074701330AE540E30E0AEA3319490158
:1089C000B3DAE900B395490133D7EC0093540901B8
:1089D000336BB70013850A0093850400EF008036DF
:1089E0009309050093850400931B090113850A0070
:1089F000EF00C03093DB0B019305050013850B00DE
:108A0000EF00002D9399090193570B01B3E7F9008B
:108A100033944C0163FAA700B387270163E627016B
:108A200063F4A700B3872701B38AA74093850400A6
:108A300013850A00EF0000319309050093850400B7
:108A400013850A00EF00802B9305050013850B00AA
:108A5000EF00002893150B019399090193D50501A7
:108A6000B3E5B90063FAA500B385250163E62501E6
:108A700063F4A500B3852501B384A5406FF09FDFA3
:108A8000B7070001130A0001E36AF9F0130A800135
:108A90006FF0DFF0E3E8D5E8B707010063FCF60408
:108AA000930BF00F33B5DB001315350033D7A60059
:108AB0009787010093870780B387E70083CB070080
:108AC00093050002B38BAB00338B7541631E0B0221
:108AD00063E4360163EACC003384CC40B386D940EA
:108AE00033B58C00B384A6401305040093850400BD
:108AF0006FF05FE3B707000113050001E3E8F6FA42
:108B0000130580016FF09FFAB3966601335D76011D
:108B1000336DDD0033D47901B395690133DC7C0119
:108B200093540D01336CBC001305040093850400BD
:108B3000B31A6601EF000021130A050093850400B3
:108B40001305040033996C01931C0D01EF00001B09
:108B500093DC0C01130405009305050013850C003C
:108B6000EF000017131A0A0113570C013367EA00CC
:108B7000130A0400637EA7003307A701130AF4FF5A
:108B80006368A7016376A700130AE4FF3307A70110
:108B9000B309A7409385040013850900EF00801AEC
:108BA000938504001304050013850900EF000015E8
:108BB000930505009304050013850C00EF00401198
:108BC00093150C011314040193D50501B365B4008A
:108BD0001387040063FEA500B385A5011387F4FF86
:108BE00063E8A50163F6A5001387E4FFB385A5013B
:108BF000131A0A01B70C0100336AEA001384FCFF60
:108C0000B3778A0033F48A00B384A5401385070044
:108C1000930504002326F100135A0A01EF00400BCC
:108C2000930905009305040013050A00EF00400AAC
:108C300013DC0A01930D050093050C0013050A00CF
:108C4000EF0000098327C100130A050093050C00FB
:108C500013850700EF00C0073305B50113D70901DD
:108C60003307A7006374B701330A9A01B7070100FD
:108C70009387F7FF935507013377F7001317070121
:108C8000B3F7F900B3854501B307F70063E6B40015
:108C9000639EB400637CF90033865741B3B7C700C5
:108CA000B385A541B385F54093070600B307F940A6
:108CB0003339F900B385B440B38525413394750148
:108CC000B3D767013365F400B3D565016FF09FC575
:108CD000130605001305000093F6150063840600D3
:108CE0003305C50093D5150013161600E39605FE4F
:108CF000678000006340050663C60506138605000D
:108D0000930505001305F0FF630C0602930610009F
:108D1000637AB6006358C0001316160093961600C7
:108D2000E36AB6FE1305000063E6C500B385C540DF
:108D30003365D50093D6160013561600E39606FE4B
:108D40006780000093820000EFF05FFB1385050051
:108D5000678002003305A04063D80500B305B0402A
:108D60006FF0DFF9B305B04093820000EFF01FF918
:108D70003305A040678002009382000063CA0500AB
:108D8000634C0500EFF09FF7138505006780020034
:108D9000B305B040E35805FE3305A040EFF01FF6E1
:108DA0003305B04067800200977701009387077E04
:108DB00083A60700177701001307077C0327070026
:108DC00023A2A600637EE500177701001307877BC7
:108DD0000325070083A50700938545006F709F9AC0
:108DE000130101FF232481002326110017770100BE
:108DF00013078779130405000325070083A50700DF
:108E000093854500EF701F9897770100938707754A
:108E100083A707006376F4009777010023A0877487
:108E20008320C10003248100130101016780000039
:108E3000977701009387877503A7070083A607002C
:108E4000832747049387F7FF2322F70483A7460469
:108E5000639407007360043067800000130101FE13
:108E6000232C8100232A910013040500938405001C
:108E700023282101232631012324410123225101EA
:108E8000232E1100EFA00F8783270400032904017C
:108E9000B7090001B3E59700930AC4002320B4008A
:108EA000930400009389F9FF370A000203270400A6
:108EB00063822A050326090013050900B3654701EB
:108EC000B37636019317560033F7E60003294900BD
:108ED00063C60700631607006FF05FFDE398E6FCCA
:108EE0009317760063D40700B3E4D400EFB0CFC883
:108EF0006FF0DFFB93C4F4FFB3F4E400232094008D
:108F0000EFA0CFB2032504008320C1010324810117
:108F100083244101032901018329C100032A81001F
:108F2000832A41001301010267800000130101FF41
:108F3000130500002326110023248100EFE0DFB891
:108F400017E7FFFF1307073A930600001306100008
:108F500093052003177501001305854AEFC00FF82C
:108F60006302050213040500EF905FFA1306050083
:108F7000130700009306000093051000130504007A
:108F8000EFC0DF87EF905FC48320C100032481001E
:0C8F9000130500001301010167800000C0
:02000004800278
:10000000F866FEFF6868FEFF0467FEFF6868FEFF93
:100010006868FEFF6868FEFF6868FEFF2C67FEFFE9
:100020006868FEFF6868FEFF5467FEFF6467FEFFB6
:100030006868FEFF7C67FEFF8C67FEFF8C67FEFF33
:100040008C67FEFF8C67FEFF8C67FEFF8C67FEFFF0
:100050008C67FEFF8C67FEFF8C67FEFF6868FEFF03
:100060006868FEFF6868FEFF6868FEFF6868FEFF5C
:100070006868FEFF6868FEFF6868FEFF6868FEFF4C
:100080006868FEFF6868FEFF6868FEFF6868FEFF3C
:100090006868FEFF6868FEFF6868FEFF6868FEFF2C
:1000A0006868FEFF6868FEFF6868FEFF6868FEFF1C
:1000B0006868FEFF6868FEFF6868FEFF6868FEFF0C
:1000C0006868FEFF6868FEFF6868FEFF6868FEFFFC
:1000D0006868FEFF6868FEFF6868FEFF6868FEFFEC
:1000E0006868FEFF6868FEFF6868FEFF6868FEFFDC
:1000F0006868FEFF6868FEFF6868FEFF6868FEFFCC
:10010000D067FEFFF867FEFF6868FEFF6868FEFFC5
:100110006868FEFF6868FEFF6868FEFF6868FEFFAB
:100120006868FEFF5868FEFF6868FEFF6868FEFFAB
:100130000865FEFF1066FEFF6868FEFF6868FEFF48
:100140006066FEFF6868FEFFD866FEFF6868FEFF17
:100150006868FEFF2067FEFFC46CFEFF306DFEFF87
:10016000D06CFEFF306DFEFF306DFEFF306DFEFF88
:10017000306DFEFF686BFEFF306DFEFF306DFEFFE1
:10018000906BFEFFA06BFEFF306DFEFFB86BFEFFB5
:10019000C86BFEFFC86BFEFFC86BFEFFC86BFEFF9F
:1001A000C86BFEFFC86BFEFFC86BFEFFC86BFEFF8F
:1001B000C86BFEFF306DFEFF306DFEFF306DFEFF41
:1001C000306DFEFF306DFEFF306DFEFF306DFEFFC7
:1001D000306DFEFF306DFEFF306DFEFF306DFEFFB7
:1001E000306DFEFF306DFEFF306DFEFF306DFEFFA7
:1001F000306DFEFF306DFEFF306DFEFF306DFEFF97
:10020000306DFEFF306DFEFF306DFEFF306DFEFF86
:10021000306DFEFF306DFEFF306DFEFF306DFEFF76
:10022000306DFEFF306DFEFF306DFEFF306DFEFF66
:10023000306DFEFF306DFEFF306DFEFF306DFEFF56
:10024000306DFEFF306DFEFF306DFEFF306DFEFF46
:10025000306DFEFF306DFEFF0C6CFEFF486CFEFF44
:10026000306DFEFF306DFEFF306DFEFF306DFEFF26
:10027000306DFEFF306DFEFF306DFEFFB46CFEFF93
:10028000306DFEFF306DFEFF3C69FEFF906AFEFFA1
:10029000306DFEFF306DFEFF206BFEFF306DFEFF08
:1002A0004C6BFEFF306DFEFF306DFEFF246DFEFFD8
:1002B000000102020303030304040404040404040D
:1002C00005050505050505050505050505050505DE
:1002D00006060606060606060606060606060606BE
:1002E00006060606060606060606060606060606AE
:1002F000070707070707070707070707070707078E
:10030000070707070707070707070707070707077D
:10031000070707070707070707070707070707076D
:10032000070707070707070707070707070707075D
:10033000080808080808080808080808080808083D
:10034000080808080808080808080808080808082D
:10035000080808080808080808080808080808081D
:10036000080808080808080808080808080808080D
:1003700008080808080808080808080808080808FD
:1003800008080808080808080808080808080808ED
:1003900008080808080808080808080808080808DD
:1003A00008080808080808080808080808080808CD
:1003B000546D725100000000546D7220537663003A
:1003C000286E756C6C2900004572726F7220696E20
:1003D00020416C745154657374207461736B732085
:1003E0000D0A00006D69616F750A00006D69616F2B
:1003F00075320A0068756E6772790A004368656332
:100400006B54696D65720000416C745F47656E5F87
:10041000546573745F517565756500004647656E78
:1004200051000000416C745F515F4D757465780038
:10043000464D754C6F770000464D754D6564000064
:08044000464D7548696768002C
:100448001000000000000000017A5200017C010148
:100458001B0D020050000000180000003878FEFF55
:100468005805000000440E507489039406990B81C6
:1004780001880292049305950796089709980A9AA5
:100488000C9B0D036C010AC144C844C944D244D32F
:1004980044D444D544D644D744D844D944DA44DB78
:1004A800440E00440B0000004C0000006C000000EB
:1004B8003C7DFEFFDC05000000440E30708903958A
:1004C8000781018802920493059406960897099873
:1004D8000A990B9A0C0370020AC144C844C944D251
:1004E80044D344D444D544D644D744D844D944DA30
:1004F800440E00440B00000050000000BC00000047
:10050800C882FEFF0005000000440E50748802896E
:10051800039305990B810192049406950796089711
:1005280009980A9A0C9B0D0320010AC144C844C9C2
:1005380044D244D344D444D544D644D744D844D9E7
:0C05480044DA44DB440E00440B000000C9
:0805DC00FC8F01000900000082
:040000058000004037
:00000001FF
